:020000040800F2
:10500000681C0020D5500008F18E00083585000886
:105010000000000000000000000000000000000090
:10502000000000000000000000000000519A00088D
:105030000000000000000000F1960008659C0008D8
:10504000E7500008E7500008E7500008E750000864
:10505000E75000082D5F0008E7500008E7500008FF
:1050600000000000E7500008015C0008E75000085D
:10507000E7500008E18A000800000000E75000083F
:1050800000000000E75000080000000000000000E1
:10509000E750000800000000E7500008E750000853
:1050A000E7500008E7500008E7500008D9A60008BC
:1050B000E7500008E7500008000000000000000072
:1050C0000348854600F0E8FC0048004781BA000824
:1050D000681C00200448804704480047FEE7FEE7BC
:1050E000FEE7FEE7FEE7FEE7019D0008C15000086D
:1050F00030B50B46014600202022012409E00D4670
:10510000D5409D4205D31D469540491B25469540F7
:1051100040191546521E002DF1DC30BDF0B51FB40C
:105120000646002082B005464024019100901BE015
:10513000019922460F46304600F098FB049A059BE1
:10514000801A994110D310461946224600F07EFB82
:10515000361A8F410197224601200021009F00F05E
:1051600075FB38184D4100902046641E0028DFDC96
:10517000019B00982946324607B0F0BD03460B4319
:105180009B0703D009E008C9121F08C0042AFAD2FD
:1051900003E00B780370401C491C521EF9D2704783
:1051A000D2B201E00270401C491EFBD270470022BF
:1051B000F6E710B513460A4604461946FFF7F0FF16
:1051C000204610BD30B504460020034600E05B1CBD
:1051D000934203D2E05CCD5C401BF8D030BDF8B503
:1051E00002464A40D40F42004B0052085B089A42E4
:1051F00002D20246084611464A0023D0C30D4A0097
:10520000DDB2120EAD1A202D35DA49020126490A07
:10521000F6058A19002C00D0524220214F1B11465E
:10522000B9402A411018C20D9A4221D0002C17D043
:10523000012D08DCDA05801AD20F8019D207DBB203
:1052400000F040FBF8BDDA05801A012340001B0680
:10525000C01880185A428018CA0F1043490007E04E
:105260004908C2071143DA05801A801940088018DE
:1052700000F020FBF8BD61000122511A001BF7E786
:105280000122D2075140AAE70122D2075040A6E7E7
:1052900070B502464A40D50F40004A00ED0740086D
:1052A0005208002814D0002A12D0C40DD30D410298
:1052B0000120C0055202490A520AE41A09181218BC
:1052C0007D34914201D3641C00E04900002C01DAD6
:1052D000002070BD0023914201D3891A0343400886
:1052E00049000028F7D100290AD0914202D10121BA
:1052F000C90705E0914201D2012101E00121C94322
:10530000E005C018401900F0D5FA70BD420005D084
:105310004200120E52428A4201DB00207047C9054A
:1053200008187047F0B507460846584087B0C00FC8
:10533000049048000E46590040084908BC1A8841AC
:1053400005D2384631461E4617460B4602465800DF
:10535000400810434CD0300D039040055900400DDB
:10536000490D0590401A0290402872DA1803012175
:10537000000B09050843019004980092002805D00D
:1053800001995242002088410092019002984021E8
:105390000A1A0199009800F059FA05460C466B4626
:1053A00007CB00F074FAC0197141039A0E0D002367
:1053B000D71756401A467A40164344D0049A002A1A
:1053C0002DD0029A012A039A15DC1205C01A9141C8
:1053D00001263605001C7141D20F059ED2070093AD
:1053E000019202962A46234600F0B2FA07B0F0BDB9
:1053F00038463146FAE71605224A0F46B218C01A57
:10540000B74101210905001C4F4100187F41114699
:1054100018187941E20F10436D19644113E0E20757
:105420006D0815436408C2071443039A0126120548
:10543000C01A91413605001C7141CE074008304327
:105440004908C01851412A46234600F074FACDE7B6
:10545000FFE7049801224000C117121A00238B4174
:1054600004983146C417381AA141EEE730B401243C
:10547000E407634030BC55E730B40124E4076140E1
:1054800030BC4FE70000E0FFF0B51FB488B00B99C7
:105490000998002448400999C00F4900490809911A
:1054A000C0070B990090490049080B910999089889
:1054B000A64608431CD00B990A98084318D00998AF
:1054C00001244000420D4800410D099824050003C5
:1054D000000B204309900B980003000B20430B9016
:1054E00050181C494018002201901446104605E04F
:1054F000002001460DB0F0BD032801DA034600E0AC
:1055000003239C46C11A0AAE0AE05F0008ADED5BBA
:105510004F00F75B7D430027AA187C41491C5B1EA6
:105520006145F2DD410004AB5A522104120C0A43DA
:10553000240C401C0828DFDB01980290009970467B
:1055400001910090059B049A0799069800F000FAD3
:10555000D0E700000DFCFFFFF0B50C465C4085B0C5
:10556000E40FE40703944C000026640859009446B5
:10557000490802460296224321D062460A431ED0C1
:105580006200570D4A000E032303550D0124024605
:105590002C492405781B1B0B360B4018234326434C
:1055A000614600901C46501AB44103D30098401C39
:1055B000009002E0921800985B41002803DA002076
:1055C000014605B0F0BD00200121090507468646C9
:1055D00011E064461D46141BB54106D36546521BB7
:1055E000B341744607430C43A646CD07400849081B
:1055F000284392185B4105460D43EAD110461843F3
:1056000013D06046194650407140084306D06046AA
:10561000101AB34106D20122002306E00022012322
:10562000DB0702E00122D2435310009874460105C3
:10563000381C6141029C039D0019694100F07BF90F
:10564000BFE70000FD03000070B54B005B0803439B
:105650000BD04B005C0D002633466542B341D41796
:10566000AD1AA34102DB0020014670BD12053018BF
:10567000514170BDC217C10F504010B54018CA0744
:105680009623002100F01EF910BD10B500229623CC
:10569000114600F017F910BD0EB5C217C10F5040EA
:1056A000CA0740180021054B0293019200910A4657
:1056B0000B4600F04DF903B000BD000033040000BC
:1056C0000EB505490291002100910A460B46019151
:1056D00000F03EF903B000BD330400004100400279
:1056E0000122400AD205090E80187F2901DA002024
:1056F0007047962903DC9622511AC84070479639A4
:105700008840704770B5CD0F4A0009030123090B8B
:105710001B0519430B4BED070024520D9A4201DA89
:10572000002070BD074B34339A4203DC9A1A00F014
:105730009DF802E00449511888402C43F1D04042C2
:1057400070BD0000FF030000CDFBFFFF4A0009030E
:105750000123090B1B051943094B10B5520D9A4241
:1057600001DA002010BD064B34339A4203DC9A1A4A
:1057700000F07CF810BD03495118884010BD0000AE
:10578000FF030000CDFBFFFFC20FD207400040081F
:105790000BD0C10D0723DB01C91840020905400ADF
:1057A0001143C2084007114370470020014670476B
:1057B00010B5002904DB0124E40740428C41214656
:1057C000002B04DB1C460123DB075242A3418B4222
:1057D00000D1824210BD000010B5002904DB012475
:1057E000E40740428C412146002B04DB1C46012388
:1057F000DB075242A341994200D1904210BD000004
:10580000CB0FDB07490010B5490802460A4307D011
:105810000A0D07240903E401090B121B002A01DC0D
:10582000002010BDC900440F0C43C100E018D20590
:10583000801800F03FF810BD0122D207002800DBDD
:10584000101A002900DB511A8142704710B5202A36
:1058500004DB0146203A9140002010BD91402023F6
:105860009C1A0346E3401943904010BD10B5202A0E
:1058700004DB0846203AD040002110BD0B46D3403F
:10588000D0402024A21A91400843194610BD10B5FB
:10589000202A06DBCB170846203A1041C1170B43DC
:1058A00006E00B461341D0402024A21A9140084341
:1058B000194610BD002904DA401C490001D14008F6
:1058C0004000704770B40024050C05D1102400047A
:1058D00002D1002921D01124050E01D10002083483
:1058E000050F01D10001241D850F01D18000A41CEA
:1058F000002801DB4000641C002908D020252E1B55
:105900000D46F540A14000D001212943084301067E
:105910001B1B000ADB1D02D5002070BC7047DB0595
:10592000181880180029F8DA401C4900F5D170BC1D
:1059300040084000704710B5002B08DA0024401CD6
:10594000614192185B411A4301D14008400010BDEB
:10595000F0B51FB482B005460C0003D0084604F031
:1059600089FF02E004F086FF2030024600902146C5
:105970002846FFF76BFF049B059A04460F46184321
:105980001143084314D0184610431BD000984021FF
:105990000A1A18460599FFF769FF05460E46009A50
:1059A00005990498FFF752FF084305D0012004E051
:1059B0002046394607B0F0BD0020C11705430E430D
:1059C0002C43374300990E986305401A7905E40A81
:1059D00000220C43FD0A0A3002D500200146E9E707
:1059E0000105101969410C9C0D9D00196941FFF7D3
:1059F000A2FFDFE7FEB500231A461B1A8A4103DB2C
:105A00000020014603B0F0BD4A000D0301212D0B1B
:105A10000905520D0D43D10702D100186D41521EE8
:105A20005110FF31FF310131002704463E46384610
:105A3000009701910246012100200905FFF716FF9A
:105A4000C3197141F818324684468E464A41614670
:105A50002846611A904104D36046241A954176463F
:105A60001F46241900986D41401C00903428E1DD48
:105A7000F91930467041091BA84103D20022D243D4
:105A8000134601E00022134601980105381C7141BC
:105A9000FFF751FFB6E70000064C0125064E05E072
:105AA000E36807CC2B430C3C98471034B442F7D33F
:105AB000FFF70AFB70C9000890C9000870B58C1880
:105AC0000578401C6B075B0F01D10378401C2A113D
:105AD00006D10278401C03E006780E70401C491C79
:105AE0005B1EF9D12B0705D40023521E0DD40B7079
:105AF000491CFAE70378401CCB1A921C03E01D787E
:105B00000D70491C5B1C521EF9D5A142D8D3002050
:105B100070BD000038B50446064805490068FFF727
:105B2000E7FA604300E0401E00900028FBD138BD3A
:105B300040420F005C010020F8B50446006881680F
:105B40008907890F012902D10168C90722D181681B
:105B5000114A10261140012500290ED181682943E0
:105B600081600120FFF7D6FF01F052F907460CE0F3
:105B700001F04EF9C01B0A2807D9606D30436065FB
:105B8000A06D2843A0650120F8BD20680068C043CF
:105B9000C007EDD10020F8BD170000801FB50B48ED
:105BA00000900B4801900B4802900B480390694607
:105BB0000A4805F055FA0A4A08481146083905F01E
:105BC0003DF900F099FB002004B010BD79C7000832
:105BD00055C70008B5C70008B3C700086801002012
:105BE0001000002010B500231A4603E0845CE3187F
:105BF0009BB2521C8A42F9D3D84380B210BD000038
:105C000010B5034800F0C0FE024800F0BDFE10BD14
:105C100004180020BC17002030B5446C1C252C4013
:105C20000125A540046C6560046863608368102BDF
:105C3000036803D099600068C26030BD9A60006854
:105C4000C16030BDF0B58BB000200790884E0A20AF
:105C500005F0B6FD7D20400105F0CCFD854C00250A
:105C6000E06B401CE06384480990FF38813808905D
:105C7000002181486171A28F0B30C270120A02723A
:105C800081740A2141727D4909788172E18C017326
:105C900045707B48099902780A74407848747649BF
:105CA0001C2000220B3105F075FE60790621484367
:105CB00000211C3005F080FE022005F0D1FD714F5F
:105CC00000210F2005F0FCFC38422064F8D0206C45
:105CD0000146401C16D048047ED58122D201002105
:105CE0000F2005F02CFE0021102005F0E9FC4106F4
:105CF000490E0022644805F019FD634F787A0228A6
:105D000002D09FE004F02AFE02225D49781DFFF7D1
:105D100059FA00287DD105F0A0FEE167A06705F0E3
:105D200089FE544A803203C20290079803910028EA
:105D30001AD101205449079054482839CB8E03804A
:105D4000098F534AFF31C33189B2A18491420BD9E3
:105D500052428918A1845B1C4D4A99B20B320180D2
:105D6000914201D300210180434B69000B33089815
:105D7000CA18017A0A91D174407A04904249107588
:105D800028394A8E68468280898EC1800422791C17
:105D9000581CFFF7F3F90198B04205DA0646694648
:105DA0000A98087504984875334803210B304172EE
:105DB0004B230299DB0403980022C91850410006C6
:105DC0000F0A0743384605F0F4FC790849000A0E2B
:105DD00008022849803100E047E0CA608860264810
:105DE000E36F1530A26F05F00DFE224880300CC81D
:105DF0002148193005F006FE1E488030C3688268CD
:105E00001D481D3005F0FEFD1B4900220B311920F5
:105E100000E017E005F0BEFD0021192005F0CCFDE3
:105E2000012005F01DFD0006000E607305D1002164
:105E30000F2005F045FC0006F9D5802200210F2037
:105E400005F07DFD6D1CEDB20A2D00D210E708486B
:105E5000864208D0002E06D00020A07302202070B9
:105E60006846808A20850BB0F0BD0A4AE6E700004C
:105E7000FFFF0100700000206114002024010020B9
:105E80003801002000D02724E8120020440100201F
:105E9000E7030000009027241449012048720A46B5
:105EA00002205E32507203203C3A507204200E3AB7
:105EB00050720F480D4B0078087022310870203165
:105EC00008770C495A1C087858714978997123331E
:105ED00018715971203318775977107551751A4612
:105EE0001E3210755175107651767047C011002022
:105EF000160100203801002010B503F07FFD20209E
:105F000003F0A6FE012005F015FB002003F0A0FE23
:105F1000044805F0B3F9044805F062FC002005F0E0
:105F200097FC10BD0001002083800000F8B503F04D
:105F30009DFE05200121000700F056FF0025144CAE
:105F4000002800D06560134E0221304600F04CFF5F
:105F5000002815D1012020700F48808F00280ED016
:105F60000127BF0200223946304600F04AFF0A20CE
:105F700004F0D4FE01223946304600F042FF65604D
:105F8000012000F069FE022000F066FEF8BD00006E
:105F90004801002000040050C00D002070470000A0
:105FA00010B5084900224A6107494B684C15234344
:105FB0004B604B68082423434B60C009C00102605A
:105FC00010BD00004C180020002002407FB50025C5
:105FD0000C460646039500F00FFEE009029003A967
:105FE00001960095684600F09FFD002804D000F05F
:105FF000D7FD002004B070BD00F0D2FD0120F9E70C
:1060000010B5002302E0C45CCC545B1C9342FAD36D
:1060100010BD000010B5214A00219069C305204839
:1060200004D54169022319434161911593699B0588
:1060300005D54369012423434361630219439369EE
:106040005B0505D54369082423434361E3011943F4
:1060500093691B0505D54369042423434361630207
:10606000194393699B0405D5436910242343436175
:106070006302194393699B0304D5446920231C439D
:10608000446119439369DB0305D5436940242343E5
:106090004361A0020143916110BD00000020024055
:1060A0004C18002070B5054600F0B2FE0646184CAC
:1060B0000AE0681C08D0002D04D000F0A9FE801B67
:1060C000A84201D9032070BDA069C007F1D1A06921
:1060D000800701D50220A061A069C00511D4A06984
:1060E00080050ED4A06940050BD4A069000508D432
:1060F000A069800405D4A069800302D4A069C0030C
:1061000003D5FFF787FF012070BD002070BD0000A0
:1061100000200240F8B51746002605460C4600F060
:106120006BFD09E029460220226800F047FD0028A7
:1061300004D1241D2D1D361DBE42F3D300F030FDC9
:10614000BE4201D20020F8BD0120F8BD10B50849BB
:1061500002460020054B497905E044001C5B94424F
:1061600003D0401CC0B28842F7D310BD7E1300207C
:106170007000002010B500F03CFE10BD10B50948BD
:1061800001F05CF880B2FFF79BFA074A074BFFF774
:106190007BF90022064BFFF7DFF9FFF7D7FA80B251
:1061A00010BD000070160020F853E3A59B843E400C
:1061B00000408F4070B50024204603F031FA474973
:1061C0004748A200641CE4B28150142CF9D346491C
:1061D00044480A7A0275497A417544490A78027638
:1061E000497841763F490520133148720A2005F06D
:1061F000E7FA7D20400105F0FDFA3A49002213310B
:106200000C2005F0C7FB00210C2005F0D5FB384819
:1062100001F014F8344C0125203C6085AD0309E001
:10622000334801F00BF880B26085218FFF392D399A
:10623000884206DB218F80B28842F1D34919884217
:10624000EED8022005F00CFB002003F0E9F9294DFF
:1062500000210F2005F034FA28422064F8D0206C89
:10626000411C38D0400435D58122D20100210F20B5
:1062700005F065FB0021102005F022FA41061948BF
:10628000490E0022C73005F051FA164DC735687A1D
:1062900005281FD102221549681DFEF793FF00282B
:1062A00018D11148AE7C66710422691C3830FEF7A3
:1062B00065FF29461331084672000D468330FEF70C
:1062C0005DFF60792946420005484A38FEF756FFCF
:1062D0000320207070BD04F041FB0000FFFF0100AF
:1062E000E01300202112002090000020380100203F
:1062F0007016002000D0272410B5144C14482246F4
:1063000010321146083904F099FD0022114BE16862
:10631000A068FFF721F9104A104B05F0BDFC0022E0
:106320000F4BFFF7A9F800220E4BFFF7ADF8FFF770
:1063300067FA206000221346E168A068FFF738FA88
:1063400001D0206810BD0020206010BD000000209A
:106350006801002000AA8F406C45D9CC955BC83FEE
:106360000000F03F40A5E54010B5084800F096FA5F
:106370000A21064800F032FA044800F01DF98005B1
:1063800003D5024800F01AF980B210BD141600209F
:10639000F8B52F4D00220121284600F032FDFFF70D
:1063A000E3FFFFF772F92B4E3146FEF771FF2A4CDF
:1063B0000122A0601146284600F023FD2749A0686D
:1063C000002588423EDB2078254F002815D0257017
:1063D000FFF7CAFFFFF759F93146FEF759FFA060F2
:1063E000FFF7D2F900223B46FFF740F800221D4B91
:1063F000FFF74AF8FFF704FA6060A068FFF7C4F9F6
:1064000000223B46FFF732F8174A184BFFF73CF8DB
:1064100006460F466068FFF7B7F9134A144B52421D
:10642000FFF732F832463B46FEF77CFFFFF7E8F90C
:1064300010496060884201DD616004E0FF21C90508
:10644000C84200D365606068FFF748F9C0B2F8BD84
:106450000004005000401B44480000200000604041
:1064600000000C4000E064403333333333B330403A
:10647000CCCCEC3F0000C842F8B505460446403598
:10648000287C0026012808D0012028742068816813
:106490008907890F01290ED101E00220F8BD0168AA
:1064A000C90708D0606D20210843606501260020DF
:1064B00028743046F8BD616DFF22013291430222FB
:1064C00011436165C1688907890F0091C168890816
:1064D0008900C1602068816892071143816000F0E3
:1064E00097FC07460EE000F093FCC01B0A2809D970
:1064F000606D0221884310210843606500202874E4
:106500000120F8BD206880680028ECDB2068C168A5
:10651000009A1143C160606D80088000401C606576
:10652000C5E70000F8B506460D464036317C012926
:106530000DD00121317401688A68520709D5416D77
:10654000202211434165002030740120F8BD022053
:10655000F8BD174B6A68D80547109A42154C8A6AED
:106560002B6812D05B035B0B1A438A6229684903CC
:1065700005D5A1680143A1600A20FFF7CBFA28687E
:10658000800312D5A06838430EE05B035B0B9A438F
:106590008A622968490302D5A1688143A1602868FD
:1065A000800302D5A068B843A06000203074F8BD15
:1065B0000110000000270140406D70470068006C2A
:1065C0007047000070B5040006D0606D26460025B7
:1065D0004036002802D006E0012070BDA565357464
:1065E000204600F0D3F8606DC00603D421688868A7
:1065F000400705D5606D1021084360653574EBE7F1
:10660000606DFF220132904302221043606588686A
:106610008207920F5B48012A02D10A68D2072BD168
:10662000032362689B079A4205D05B429A4202D0DC
:106630005B009A4209D10A69920092080A612168B6
:106640000A6963681A430A610CE00A6992009208B9
:106650000A6181680F2292049143816081686268B7
:10666000114381602168CA6818239A43CA6021686F
:10667000CA68A3681A43CA6081680122520691431E
:1066800081608168A28E5206114381602068816812
:10669000C90004D481680122120711438160206877
:1066A000C168394A1140C1602069E168022825D0DB
:1066B00000200143204620300278037B52035B0018
:1066C0001A431143226B1143A26992031143E269F9
:1066D000D20311432268D3681943D160616A0A4624
:1066E000FF3AC23A05D0A26A11432268D36819431F
:1066F000D16042780121012A02D00BE00420D8E7C2
:106700000078002823D0606D202210436065A06DC2
:106710000843A065E06B012820681FD00169C90704
:1067200003D0016949084900016120684169C9082D
:10673000C900416120684169A26B11434161A565AF
:10674000606D80088000401C6065002070BD20687E
:10675000C26801231B041A43C260DBE70269FF23FE
:106760009B009A43026120680269236CA66C1A435D
:10677000636C33431A430261206802690A43026171
:10678000D3E70000002701401902FEFF10B586B0D4
:10679000044614216846FEF70AFD0E492068884227
:1067A00016D10D48416B421511434163C16A012264
:1067B0001143C162C06A69461040059002200090F2
:1067C00003200190002002900520000700F050FAFD
:1067D00006B010BD0024014000100240F8B5044688
:1067E0004069254640350E4608280BD02068C06811
:1067F000C00709D0606D202108436065002028741F
:106800000120F8BD082700E00C2700F001FB0090F4
:1068100011E0701C0FD0002E05D000F0F9FA00999D
:10682000401AB04207D9606D04210843606500201A
:1068300028740320F8BD206800683842E9D0606DF4
:1068400001214902084360652068C16809058A0F73
:106850000C21002A1BD12022125D002A17D10268C8
:10686000120714D5826853070122002B08DB436806
:106870008B434360606D130298431043606506E0EC
:10688000606D202318436065A06D1043A065A0696A
:10689000002801D1206801600020F8BD70B50446D1
:1068A000216800208968490721D425464035297C84
:1068B00001291CD001212974E169012904D0204655
:1068C000FFF73AF9002811D1616D0A4A1140FF2201
:1068D0000132114361650021A165297422681C21E0
:1068E000116021688A6804231A438A6070BD0220FF
:1068F00070BD0000FEF1FFFF30B5014620314A793E
:106900000023022A04D00422C2630B71012030BD8F
:10691000026814680E25AC431460026814686408A9
:1069200064001460446C1C22144001221546006C63
:10693000A54045604A7118460B7130BD70B5002402
:10694000014620314A79022A03D00421C16301247F
:1069500018E0026813680E25AB43136002681368E1
:106960005B085B001360436C1C2213400122154638
:106970009D40036C5D604A7100220A71816B0029A1
:1069800000D08847204670BDF0B4016C0D680168E6
:106990000C68466C1C2304221E401746B7402F4249
:1069A0000ED067070CD50C68A40602D40C6894437B
:1069B0000C60416C19408A40016C4A60016B1AE01E
:1069C0000227B74002462F402032002F17D0A707DA
:1069D00015D50C68A40605D40C680A25AC430C60D8
:1069E00001215171446C02211C40036CA14059608B
:1069F00000211171C16A002918D0F0BC084708278E
:106A0000B7402F4212D0240710D50C680E25AC4396
:106A10000C60446C01211C400B46A340046C636075
:106A2000C163517100211171416BE4E7F0BC704703
:106A300070B504003CD01F48256814212818FEF7C3
:106A400057FB800060641C482064022120462030EF
:106A50000246417129681948E3680140A0686669E7
:106A60001843236933431843A3691843E369184360
:106A7000236A1843084328600121A06889038842DB
:106A800010D00D488030836A656C1C210D400F26A4
:106A9000AE40B3438362656C63680D40816AAB406E
:106AA0000B4383620020E06301215171107170BDBE
:106AB000012070BDF8FFFDBF000002400F80FFFF06
:106AC000F8B504468C46203001790025012909D00B
:106AD0000126067141790027012905D00771022599
:106AE0002846F8BD0220F8BD02214171E763206805
:106AF000016849084900016061462046FFF78CF8AB
:106B0000206B00282068016801D00E2205E00422D5
:106B100091430160206801680A22114301602068E6
:106B2000016831430160DBE7F8B51A4E0546307C59
:106B30000F46012807D0012030741748FFF7B2FA3A
:106B4000010002D021E00220F8BD0020C0433860DF
:106B50006C6814E02046FFF723FA0F48FFF7A2FA0B
:106B600001460E48426808239A4342604268431532
:106B70009A434260002901D03C6006E08034A86856
:106B80006A68C0018018A042E4D80020307408462A
:106B9000F8BD00004C18002050C300000020024047
:106BA00005484168022211434160416801221143B6
:106BB000416000207047000000200240F8B50C4CF6
:106BC0001646207C0F46012808D001202074094871
:106BD000FFF768FA0025002802D006E00220F8BD81
:106BE00065613E600348FFF75DFA2574F8BD00005B
:106BF0004C18002050C3000011484168C9070BD051
:106C0000EFF3108172B60F4AC2600F4AC26081F37F
:106C100010884168C9070ED1416889070DD5EFF387
:106C2000108172B6094A0261094A026181F3108833
:106C30004068800701D501207047002070470000A0
:106C400000200240EFCDAB8905040302BFAE9D8C4E
:106C5000161514137047000010B504494A69024222
:106C600002D04861FFF7F6FF10BD000000040140AC
:106C7000FCB500230124A2E027462A469F403A4063
:106C80006FD04D68012D05D0022D03D0112D01D0FC
:106C9000122D16D185680326AC465D00AE46AE4087
:106CA0006546B543AC46CE687546AE4065462E4354
:106CB000866046680D79BE43ED06ED0F9D40354375
:106CC0004560C6685F000325BD40AE46AE4335460D
:106CD0008E68BE402E43C6604E68022E01D0122E32
:106CE00014D1DE08B60036180196366A5D07B44640
:106CF000EE0E0F25B54000966646AE43B4460D69CC
:106D0000009EB54066462E43019D2E62066875467C
:106D1000AE430D79AD07AD0FBD40354305604D68FD
:106D2000ED004BD5294D6E6B26436E639E08284DB2
:106D3000B6007519AC46AD689E07360F0F27B740F1
:106D4000BD4305273F07B84201D1002715E0214F79
:106D5000B84201D1012710E01F4FB84202D10227EB
:106D60000BE02BE01D4FB84201D1032705E01C4F7B
:106D7000B84201D1052700E00627B7402F436546FA
:106D8000AF60184D2E684F689643FF0300D5164339
:106D90002E606E684F689643BF0300D516436E6041
:106DA000AE684F689643FF0200D51643AE60EE68AA
:106DB0004F689643BF0200D51643EE605B1C0A681D
:106DC0001546DA4000D057E7FCBD00000010024035
:106DD000000001400004005000080050000C00506A
:106DE000001C0050000401400069084000D0012050
:106DF0007047426913460B401B0491430B43836168
:106E00007047002A01D0816170478162704700009D
:106E100001488068704700005001002002488168E6
:106E200002788918816070475001002010B5084829
:106E300000240168402211430160204600F00AF856
:106E4000002801D0012401E000F042FA204610BDE4
:106E50000020024070B504460D4D7D202978C00009
:106E6000FEF746F901460B480068FEF741F900F0CD
:106E70002BFF002809D1042C07D200222146401EF6
:106E800000F04EFA00206C6070BD012070BD000063
:106E9000500100205C01002070477047F8B502F0F7
:106EA000E5FE604C0120E070208AFEF7EEFB014613
:106EB0007F20C005FEF7ECF95B4D06462968FEF71A
:106EC0008EF928600120A16AC005814201DA0846D6
:106ED00003E03046FEF7D8F9A062FF21C90500257E
:106EE000C84200D3A562607800280BD102214F4828
:106EF000FFF77AFF02004E494E4817D00022FFF7F5
:106F000080FFE56202214948FFF76EFF4A4E0028E4
:106F100055D0E562B08AFEF7B8FB434F3968FEF7FB
:106F20008BFC5FD24549012008705DE00122D1034E
:106F30004048FFF766FF208AFEF7A7FB01467F2047
:106F4000C005FEF7A5F9E16AFEF749F93C49E062A0
:106F50008842D7DD38480127F926403000900A21C1
:106F60003046FEF7C5F8002903D131493148FFF713
:106F700001F902212D48FFF737FF002801D0002733
:106F800001E0002F12D102212848FFF72DFF002831
:106F90000CD104F049FE00990120888005F0A0FB87
:106FA000642003F0BBFE28492648C8600A2003F08D
:106FB000B5FE3046761EF6B20028D0D1A2E7208A70
:106FC000FEF763FB01467F20C005FEF761F9E16A29
:106FD000FEF705F91D49E06288429BDB1A49194812
:106FE000C86097E715480570708F401EFEF742FB9A
:106FF0003968FEF721FC06D82079002803D014490F
:107000000120087001E012480570708FFEF73DFB0B
:107010003968FEF711FC04D22079002801D004F071
:10702000C5FDF8BD140100204C01002000040050F3
:107030000080000000000050C00D002076000020FD
:10704000000040400400FA0500ED00E00000A04010
:1070500087000020704770B5040010D0022025463C
:107060002035A873204601F043FDA87B032805D0F6
:10707000204600F0B9F80020A873687370BD0120A5
:1070800070BD7047704710B5044600680168C94379
:10709000C90708D18168C943C90704D101214160EA
:1070A0002046FFF7FBFE20680168C943890708D422
:1070B0008168C943890704D4022141602046FFF753
:1070C000EBFE20680168C943490708D48168C943B9
:1070D000490704D404214160204600F0F7F82068F5
:1070E0000168C943090708D48168C943090704D462
:1070F000082141602046FFF7ADFF20680168C943C1
:10710000C90608D48168C943C90604D41021416066
:107110002046FFF7C2FE20680168C943890608D4EB
:107120008168C943890604D4202141602046FFF7C5
:10713000A9FF20680168C943490608D48168C9438A
:10714000490604D4402141602046FFF79AFF10BD54
:10715000F8B5040005D025462035A87B002802D0CC
:1071600006E00120F8BD00206873204600F04EF8CC
:107170000220A8732068C26884466368012B01D18D
:107180000620824316486169814202D007204003ED
:107190008243002B01D1D82082431248A6680240C6
:1071A00018463043676A266A3E433043A66A304336
:1071B0001043002B02D0012B04D005E02369E269C3
:1071C0001A4300E0E2681043054A914202D0A269E6
:1071D000114308436146C8600120A8730020F8BD30
:1071E000FFFF0000F8F119FF10B50068054988425B
:1071F00007D10548816B4900490881630D2000F0E3
:1072000073F810BD007C00400010024010B500680B
:10721000084988420CD10848816BC204114381633C
:10722000002201210D2000F07BF80D2000F06CF809
:1072300010BD0000007C0040001002400068C069E2
:1072400070470000F8B50446022025462035174651
:10725000A8731D480268C3041A4302602068C2680C
:107260009B121A43C2602068026901263243026100
:10727000226810205060206881611021204601F0B2
:10728000A7FC03281FD021680820486020684761B8
:107290000821204601F09CFC032814D0204601F070
:1072A00027FCA87B03280ED02068816831438160C9
:1072B000206801693143016120680169042211439A
:1072C0000161AE730020F8BD00040140704700006A
:1072D0000448416B012211434163816B0204114355
:1072E0008163704700100240002809DBC106C90E07
:1072F0000120884003490860BFF34F8FBFF36F8FB1
:107300007047000080E100E0002805DBC106C90EDF
:1073100001208840014908607047000000E100E05A
:1073200010B503F0F9FA10BD02494A6882434A6079
:107330007047000000700040024801688215114348
:10734000016070470070004002494A6802434A6089
:107350007047000000700040054801680222114398
:1073600001600448016904221143016130BF704784
:107370000070004000ED00E0F0B5154A1368154DAF
:1073800054152D6A2340ED07ED0F002B04D0002D7E
:1073900002D01668A64316601668B608B600064303
:1073A00016600D48076904263743076101290DD08F
:1073B00040BF20BF20BF0169B1430161002B04D051
:1073C000002D02D0106820431060F0BD30BFF2E7FE
:1073D000007000400000014000ED00E0F8B50446F8
:1073E00000780027534D800671D5524E403EB06B59
:1073F000C00004D4B06BA9050843B06301274E4810
:107400000168C90511D40168821511430160FFF7B5
:10741000FFFC009005E0FFF7FBFC0099401A642890
:1074200037D845480068C005F5D5326803210905FD
:1074300060680A400140914208D08103890F032906
:1074400004D13168890301D50120F8BD2A690321DF
:1074500009040A4022D0084090421FD020788006BC
:107460001CD528692A6988430121C9040A432A6175
:107470002A698A432A612861C0050FD5FFF7C8FC35
:10748000009008E0FFF7C4FC0099411A2B488142A4
:1074900001D90320F8BD28698005F3D56168880308
:1074A000800F032805D132680005824301400A435A
:1074B0003260286903226168120411400843286180
:1074C000002F04D0B16B012000078143B163207805
:1074D000C00705D0E868A168800880000843E8601C
:1074E0002078800705D5E8680C218843E1680843C7
:1074F000E8602078400706D5E868032189028843C0
:1075000021690843E8602078000706D5E868032170
:107510000903884361690843E8602078000606D5BE
:10752000E868032189048843A1690843E8600020D2
:10753000F8BD0000401002400070004088130000B9
:10754000F8B50E46050038D05E480068C007C00F89
:10755000B04214D25B4C20684008400030432060A9
:10756000FFF756FC074605E0FFF752FCC11B5648E3
:1075700081427AD82068C007C00FB042F4D1287881
:10758000524C800705D5E068F0218843A96808437C
:10759000E0602878C00752D06868022806D0032827
:1075A00007D0216801280AD0890504E021688903F1
:1075B00001E021688901002903DB0120F8BD4907AA
:1075C000F9E7E168890889000143E160FFF720FCE1
:1075D0000746686802280AD0032814D001281ED064
:1075E00029E0FFF715FCC11B374881423DD8E06810
:1075F0000007800F0228F4D121E0FFF709FCC11B2E
:107600003148814231D8E0680007800F0328F4D167
:1076100015E0FFF7FDFBC11B2B48814225D8E06830
:107620000007800F0128F4D109E0FFF7F1FBC11B2F
:107630002548814219D8E0680007800FF5D121481C
:107640000168C907C90FB14217D901684908490043
:1076500031430160FFF7DCFB074608E005E0FFF778
:10766000D7FBC11B1848814201D90320F8BD15483A
:107670000068C007C00FB042F1D12878400706D596
:10768000E068072109028843E9680843E060287838
:10769000000707D5E0680721C90288432969C900A6
:1076A0000843E06000F03AF8E168094A0906090F6A
:1076B000515CC8400749086007480068FFF7CAFBEB
:1076C000F8BD0000002002408813000000100240B6
:1076D000BAC800085C010020540100200448054994
:1076E0000068C968044A4905490F515CC8407047A1
:1076F0005C01002000100240D3C80008044805497E
:107700000068C968044A8904490F515CC840704741
:107710005C01002000100240D3C8000870B51A4A6E
:10772000D3681A490C2018408D0004280CD04E0054
:10773000082810D00C2810D050680004410F0120F8
:10774000C003491C884070BD1068C00601D50846BA
:1077500070BD284670BD304670BD98020C4C000FBD
:10776000205C1B029C0FD368641CDB0301D53146EF
:1077700003E01268D20600D4294603F092F82246AC
:107780000023FDF7CBFC70BD0010024000093D0056
:10779000CAC80008FEB505007ED0FE4CE7680C2084
:1077A000E66807400120000406402878C00747D05B
:1077B000082F05D00C2F0AD101200004864206D1E3
:1077C000206880033CD568680028E5D038E00120B7
:1077D00069680004814203D121680143216011E0FE
:1077E000052301221B0492049942216802D111430E
:1077F0002160F1E781432160216801400091206808
:1078000090432060686800280DD0FFF701FB0090CE
:1078100005E0FFF7FDFA0099401A64287BD820683C
:107820008003F6D50CE0FFF7F3FA009005E0FFF7D0
:10783000EFFA0099401A6428F0D820688003F6D443
:107840002878800756D50923E868042F0DD00C2F1F
:1078500001D1002E09D000283CD021689943014372
:107860002160FFF7D5FA064628E02168490701D5CF
:10787000002891D061681F22120291432A691202E6
:10788000114361602168994301432160FFF746FF7E
:10789000E16809060A0F00E08BE1BF49895CC84036
:1078A000BE490860BE480068FFF7D4FA002873D1CB
:1078B00020E0FFF7ADFA801B0228AFD82068400710
:1078C000F7D560681F210902884329690902084326
:1078D00060600FE02068400840002060FFF798FAE1
:1078E000064604E0FFF794FA801B022896D8206829
:1078F0004007F7D42878C00660D5002F0CD0A869BF
:1079000000284AD02068FF21013108432060FFF79A
:107910007FFA06462EE0C1E02068800502D5A869FE
:107920000028A6D06068072149038843296A0843D4
:1079300060606068297F0002000A090608436060F1
:10794000286A410B0120C003491C8840E1680906F0
:107950000A0F9149895CC8409049086090480068C6
:10796000FFF778FA002817D128E0FFF751FA801BBB
:107970000228A2D820688005F7D56068072149034E
:107980008843296A084360606068297F0002000A12
:1079900009060843606011E0E2E02168FF20013041
:1079A00081432160FFF734FA064604E0FFF730FA1E
:1079B000801B022872D820688005F7D42878794E79
:1079C000000724D568690028306910D001210843D8
:1079D0003061FFF71DFA009005E0FFF719FA0099F2
:1079E000401A02285AD830698007F6D50FE04008BF
:1079F00040003061FFF70CFA009005E0FFF708FA4D
:107A00000099401A022849D830698007F6D42878AE
:107A1000400766D500200290A06BC00006D4A06B82
:107A2000012109070843A063012002905E48016814
:107A3000C90511D40168821511430160FFF7E8F907
:107A4000009005E0FFF7E4F90099401A642825D872
:107A500055480068C005F5D5FF20AA68013082426C
:107A600003D131690143316111E001218902002A0A
:107A700007D005231B029A4203D132690A433261BF
:107A8000EFE7326982433261306988433061A86828
:107A9000002810D0FFF7BCF9009008E05FE0FFF786
:107AA000B7F901460098091A4048814257D8306911
:107AB0008005F4D50DE0FFF7ABF9009006E0FFF785
:107AC000A7F90099411A3948814248D830698005A0
:107AD000F5D40298002804D0A06B0121090788433F
:107AE000A063686A002866D00C2F3ED001263606B7
:107AF0000228206805D0B0432060FFF789F90546C9
:107B00002FE0B0432060FFF783F9074604E0FFF75A
:107B10007FF9C01B022822D820688001F7D4E96AC7
:107B2000A86AE2680843296BFD231B049A431143AA
:107B30000843E060206830432060FFF769F905469C
:107B400004E0FFF765F9401B022808D8206880018F
:107B5000F7D530E0FFF75CF9401B022801D903207C
:107B6000FEBD20688001F5D425E00128F8D0E0684A
:107B700001210904AA6A014091421AD10F21890406
:107B8000EA6A0140914214D1032189050840296B1A
:107B900088420DE000100240BAC800085C010020D5
:107BA0005401002040100240007000408813000083
:107BB00001D00120FEBD0020FEBDF8B504000ED0AE
:107BC000FF27606A0537002500280AD02561656116
:107BD00026464036A562707C002807D00AE00120C6
:107BE000F8BD6068B842F3D0E561F1E7357420462E
:107BF00000F03EF8022171742068026840239A4325
:107C000002602123A26860689B021A40384010433A
:107C1000E3688A021340184323690B40217D18430F
:107C2000C907C90F0843A169931019400843E169C6
:107C3000382319400843216A802319400843A16A68
:107C400093001940084321680860A0690421000CD2
:107C50000840616A10231940084321684860206881
:107C6000C1699143C1616565012070740020F8BD50
:107C700010B586B0044614216846FDF798FA1049FD
:107C80002068884219D10F48416B82141143416327
:107C9000C16A01221143C162C06A002110400590EF
:107CA000E0200090022001900320039002910491B3
:107CB000052069460007FEF7DBFF06B010BD000097
:107CC0000030014000100240094910B5401E8842B2
:107CD00001D9012010BD074C60610321081F02F08B
:107CE0001BFE0020A06107202061002010BD0000C5
:107CF000FFFFFF0000E000E0F0B502462032137EF7
:107D0000012B1ED001251576022353760668746870
:107D1000B3687027BC430F68274377600068AC07DF
:107D2000A04205D0084CA04202D0084CA04204D189
:107D300080244968A343194381605576002010765A
:107D4000F0BD0220F0BD0000000801400014014019
:107D500070B5050005D02C462034607E002802D086
:107D600006E0012070BD00202076284600F010F8C3
:107D700002206076291D286801F0EEFF0120A0771F
:107D8000A076E076207760776076002070BD0000F6
:107D9000006801218907884204D10348816B0122D0
:107DA000114381637047000000100240F8B505469A
:107DB00004462035287E012817D001262E76022081
:107DC0006876226890687727FF23B8431B029843A0
:107DD00090600A68502A31D00EDC202A4BD006DC95
:107DE000002A48D0102A3AD145E00220F8BD302AB6
:107DF00041D0402A33D136E0602A27D0702A12D0F1
:107E000001200003121A2AD0824228D1CB684A6886
:107E10008968206801F0D9FF2068816801229203F7
:107E2000114381601BE0CB684A688968206801F0D3
:107E3000CCFF216888683843886010E0CA684968C8
:107E4000206802F03CF85021206806E0CA684968C2
:107E5000206802F045F86021206801F0C1FF6E76CD
:107E600000202876F8BDCA684968206802F027F823
:107E700040212068F1E711462068EEE710B586B092
:107E8000044614216846FDF792F90121206889070C
:107E9000884212D10A49CA6A02200243CA62C96AE8
:107EA000019001400591410200910021029103914E
:107EB000049069460348FEF7DBFE06B010BD0000E3
:107EC0000010024000040050F8B506460446203673
:107ED000307E0D4601280BD0012008273076002A7D
:107EE00008D0042A16D0082A2AD00C2A4DD137E00F
:107EF0000220F8BD206801F07BFF206881693943CA
:107F000081612068816904229143816120688169CF
:107F1000EA6812E0206801F083FF2068816901228D
:107F2000D2021143816120688269012189028A435A
:107F3000826120688169EA6812021143816124E04C
:107F4000206801F086FF2068C1693943C16120685B
:107F5000C16904229143C1612068C169EA6812E0E5
:107F6000206801F091FF2068C1690122D20211430B
:107F7000C1612068C269012189028A43C261206807
:107F8000C169EA6812021143C16100203076F8BD70
:107F900070B5050005D02C462034607E002802D044
:107FA00006E0012070BD00202076284600F00FF882
:107FB00002206076291D286801F0CEFE0120A077FE
:107FC000A076E076207760776076002070BD7047FD
:107FD00070B505462C4602202034002908D004291B
:107FE0000BD008290ED0627F012A10D0012070BD6D
:107FF000A27E012AFAD1A0760AE0E27E012AF5D11A
:10800000E07605E0227F012AF0D1207700E060775A
:108010000122286801F0CCFE012228689207012184
:10802000904205D0074A904202D0074A904204D1BC
:1080300082685207520F062A02D002680A43026081
:10804000002070BD000801400014014070B50446D6
:108050000D460068002201F0ABFE2068016A0C4A60
:10806000114203D101684908490001600120203410
:10807000002D06D0042D06D0082D06D060770020F4
:1080800070BDA076FBE7E076F9E72077F7E7000020
:10809000111100007047704770470000F8B5026882
:1080A0000446D06911689668814B05461D4020231F
:1080B000002D6CD0F7077F4DFF0FBC460D402F43BE
:1080C00079D02546C7078035002F06D0CF0504D5C7
:1080D000012717622A683A432A60820708D5F20707
:1080E00006D0276802223A622A6804273A432A60A7
:1080F000420708D5F20706D02668042232622A68B1
:10810000022632432A6002070AD50A461A4066460A
:10811000324305D02668082232622E6816432E604C
:10812000020508D54A0106D501222668D20232622C
:108130002A681A432A602A68002A30D0800606D5A9
:10814000880604D5616E002901D02046884728683A
:1081500021688968490602D42821084225D0204692
:1081600002F0D1F820688168490619D5826840215B
:108170008A438260206F002812D04F498163206FAC
:10818000FEF7DCFB00280AD0206F816B06E0850635
:1081900011D58D060FD5616E77E020468847F8BD72
:1081A0002046FFF779FFF8BD05E02046FFF774FF92
:1081B00000202860F7E7256E012D56D1C50654D55D
:1081C000CD0652D5102616622068816825464906DC
:1081D000403500292ADA226F116849680904090C20
:1081E000E1D02F8B8F42DED9698311680968890637
:1081F00017D4016832019143016020688168490801
:108200004900816020688168402291438160E36772
:108210000020206620680168B1430160206FFEF7EE
:108220006BFB288B698B401A81B21AE0298B6A8B11
:10823000891A6A8B89B2002AB5D00029B3D00268A6
:10824000FF252135AA430260206882685208520047
:108250008260E36700202066606620680268B2439F
:1082600002602046FFF716FF9DE7C50208D575029C
:1082700006D50120000510622046FFF70CFF92E7AB
:10828000050605D50D0603D5A16E002985D18AE71F
:10829000400688D5480686D5116820464024A1436B
:1082A000116083670021816600F043F97BE70000DD
:1082B0000F080000200100042DA2000810B50400E2
:1082C00003D0A06F002802D007E0012010BD0021DC
:1082D00074200155204600F027F82420A06720686C
:1082E0000168490849000160204602F05FF8012852
:1082F000ECD0606A002802D0204601F081FE2068A0
:1083000041680922D20291434160206881682A2293
:108310009143816020680168012211430160204679
:1083200001F0D4FE10BD0000F0B587B00646142160
:108330006846FCF73CFF2C493068884251D12B48F5
:10834000416B0122920311434163C16A012211432F
:10835000C162C06A002510400590032040020090D1
:108360000220032701A9A1C1042004900520694629
:108370000007FEF77DFC1F4C1D48A560E56081C429
:108380008027E560A7602020256160610002A06170
:108390001848083CFEF74CFB002801D0FDF7FEFD15
:1083A0003467A662144C124821461438206003201A
:1083B000606010200831A1C16561A561E5612046BA
:1083C0002562FEF735FB002801D0FDF7E7FDF466D6
:1083D000002201211B20A662FEF7A2FF1B20FEF750
:1083E00093FF07B0F0BD00000038014000100240CC
:1083F00030000240BC1700200418002070B5C36F85
:10840000202B27D100290BD0002A09D00124836812
:108410002403A34206D10369002B03D1CB0701D06B
:10842000012070BD034660331C7D012C12D0012455
:108430001C7500230366084C0368A34207D05C68E0
:10844000240204D51C680125AD062C431C6002F0F3
:10845000ADF870BD022070BD004800407047704705
:10846000FFB50446806F83B017460D4620285ED1C5
:10847000002D0AD0002F08D0A168C001814207D189
:108480002069002804D1E80702D0012007B0F0BD20
:10849000204660300090007D012848D000980121DE
:1084A00001750020802108512120A067FEF7B0FC53
:1084B000264640360190378277820120A16800036A
:1084C000814202D12069002805D02F46002500995D
:1084D0000020087511E00027F9E7002280212046DE
:1084E00002F0AAF8002815D1002F15D0216838789D
:1084F00088627F1C708A401E7082708A019B0028EF
:1085000006980090E9D100224021204602F094F81C
:10851000002808D00320B9E728882168C005C00DCD
:108520008862AD1CE6E72020A0670020AEE70220AD
:10853000ACE77047034D044C04A002F091F9E560EC
:10854000FAE700000400FA0500ED00E048617264FB
:108550004661756C745F48616E646C65722E0D0ABD
:108560000000000000B585B014216846FCF71FFE2E
:1085700004490220C8800449488300F053FC05B038
:1085800000BD0000000E00201401002010B50524DD
:108590002407002204212046FEF733FC0022082194
:1085A0002046FEF72EFC0A2002F0BFFB0122042128
:1085B0002046FEF726FC0A2002F0B7FB0022042129
:1085C0002046FEF71EFC10BD10B50524240700222E
:1085D00004212046FEF715FC012208212046FEF763
:1085E00010FC0A2002F0A1FB012204212046FEF724
:1085F00008FC0A2002F099FB002204212046FEF725
:1086000000FC10BDF8B500240526074625463607B0
:10861000002204213046FEF7F4FB0A2002F085FB1D
:10862000012204213046FEF7ECFB6006040E08210F
:108630003046FEF7D9FB002801D0641CE4B20520C7
:1086400002F073FB6D1CEDB2082DE1D3002F03D0B7
:10865000FFF79CFF2046F8BDFFF7B6FFFAE770B5BD
:10866000052605463607002204213046FEF7C9FBE1
:108670000024E80901D0012200E000220821304650
:10868000FEF7BFFB6806050E0A2002F04EFB012232
:1086900004213046FEF7B5FB0A2002F046FB00221B
:1086A00004213046FEF7ADFB0A2002F03EFB641CBD
:1086B000E4B2082CDDD370BD10B5052424070122D7
:1086C00008212046FEF79DFB012204212046FEF7EB
:1086D00098FB002208212046FEF793FB0A2002F0B7
:1086E00024FB002204212046FEF78BFB10BD10B5B1
:1086F00005242407002204212046FEF782FB0022E5
:1087000008212046FEF77DFB0A2002F00EFB012225
:1087100004212046FEF775FB012208212046FEF7C2
:1087200070FB0A2002F001FB10BD70B505252D0776
:108730000024012208212846FEF763FB062002F0F0
:10874000F4FA012204212846FEF75BFB062002F022
:10875000ECFA07E0641CE4B2FA2C03D9FFF7C7FF78
:10876000012070BD08212846FEF73EFB0028F1D10C
:10877000002204212846FEF744FB002070BD0000C3
:10878000F8B501F0D5FC01F005FD5B480068C06953
:10879000FDF7F4FC594C5A49A082898F594E0025A7
:1087A000002931D0A26A730357499A4202DB0222A0
:1087B0000A7000E00D700A7801218902002A05D0B4
:1087C000012A0ED0022A10D0032A1DD1608B012865
:1087D0002ED0022818D1484808214038FFF736FC2F
:1087E00012E0FF22F5329042F0D2608B01281DD0BA
:1087F000022804D008E03046FEF703FB04E03E48C0
:1088000008214038FFF7E4FBFDF7C2FD207001218D
:10881000C9023046FEF7E8FA0127FF0300282DD0F1
:108820003A480560A079002804D007E00022E2E77A
:108830000122E0E70120A07101F07AFF802130469B
:10884000FEF7D2FA002806D0002208213046FEF7B3
:10885000D8FA012205E0012208213046FEF7D1FABC
:108860000022052039460007FEF7CBFA244C284E9B
:108870004034A08C274F012803D01CE0A5710022B2
:10888000EAE725486946088072B680212348FDF74B
:108890009DFB002804D0022269462048FDF73AFCDF
:1088A00062B61FA001F0DCFFA58403F019FF64206D
:1088B00002F034FAFE60608C012808D1104865840B
:1088C000058003F00DFF642002F028FAFE60208C82
:1088D000012806D1258403F003FF642002F01EFA6C
:1088E000FE600748124A0188914202D1C0880028E0
:1088F00000D1FE60F8BD00003817002014010020F0
:10890000C00D002000040050850000204C01002014
:108910000400FA0500ED00E0AAAA0000384A0008A9
:10892000BDF8C8EBC9FDBCB6C4A3CABD0D0A0000A2
:10893000AA55000038B500246946202000F0AAF8A6
:1089400068460078572800D001246946212000F0AD
:10895000A1F868460078032800D001246946222047
:1089600000F098F868460078402800D00124694655
:10897000232000F08FF868460078082800D00124F2
:108980006946302000F086F868460078AA2800D0B2
:1089900001246946322000F07DF80C486946008FBA
:1089A0000978884200D001246946332000F072F82B
:1089B00006486946403040880978884201D1002C39
:1089C00002D004490248C86038BD0000C00D002034
:1089D0000400FA0500ED00E038B55721202000F032
:1089E0007AF80321212000F076F84021222000F0BF
:1089F00072F80821232000F06EF8AA21302000F040
:108A00006AF81048018F142901D8002901D10121E9
:108A100001870C4C40346188142901D8002901D108
:108A200002216180008FC1B2322000F054F8A17899
:108A3000332000F050F8684600F006F80A2002F0F3
:108A400074F938BDC00D002010B501460F2000F0AC
:108A500021F8002800D0012010BD10B50446FFF712
:108A60002BFE3220FFF7FBFDFFF75FFEE0B2FFF7C2
:108A7000F6FDFFF75AFEFFF71FFE3320FFF7EFFD6D
:108A8000FFF753FE0020FFF7BDFD0446FFF72FFE62
:108A9000204610BD10B50C46FFF7DFFF2070012007
:108AA00010BD70B50D460446FFF706FE3220FFF7F5
:108AB000D6FDFFF73AFEE0B2FFF7D1FDFFF735FE36
:108AC0002846FFF7CCFDFFF730FEFFF710FE0A2027
:108AD00002F02BF970BD10B5FFF7E3FF012010BDC8
:108AE00010B50248FEF7CFFA10BD00007016002046
:108AF000FEB50446002772B6334A01688B1804D1CC
:108B00003248C76803208004074088680190C8681D
:108B1000009048698E69002B08D12C4940398B6A36
:108B2000CD042B438B628B6AAB438B62014631438E
:108B30003CD025492368CB4205D12449CA68032388
:108B40009B049A43CA6025462035002810D021682E
:108B50000A6901231A430A612168486108212046F5
:108B600000F036F8032800D1A87321680820486077
:108B7000002E10D020680169012211430161206894
:108B800086611021204600F023F8032800D1A87345
:108B90002168102048600C482168C14206D10B486A
:108BA000C1680322920491433943C160206801697E
:108BB000490849000161216801988860216800988E
:108BC000C86062B6FEBD00000084FFBF40100240D6
:108BD00070B506460B480D46002409490068FCF7AD
:108BE00087FA7D21C90048433168401E00D1032423
:108BF0000B682A469A4301D00028F6D1204670BD62
:108C0000204E00005C0100201CB500211648009198
:108C1000144A01910260C16312054260816007221B
:108C20008263012202610246C16020321170FF237B
:108C30005170C23343628162117301638161042206
:108C400041634261C161FDF7BDFC0848009080139B
:108C5000019069460448FDF765FC00210248FDF7D4
:108C60000BFC1CBD0024014014160020020000046F
:108C700008B50848016B012211430163006B012113
:108C80001040009000220A20FEF74AFB0A20FEF75F
:108C90003BFB08BD00100240F0B587B014216846C8
:108CA000FCF785FA4748C26A04210A43C262C26AD5
:108CB0000A400592C16A80263143C162C16A3140CF
:108CC0000591C16A01242143C162C16A2140059115
:108CD000C16A02252943C162C06A22462840059024
:108CE00005201C210007FEF78CF801223649374881
:108CF000FEF787F8002236493448FEF782F89121C2
:108D00000520002209020007FEF77BF83148019098
:108D1000002705206946029700940007FDF7A8FF89
:108D20000C20009011200190032003900520029751
:108D300069460007FDF79CFF10206A46039591C223
:108D4000052069460007FDF793FF11200190029767
:108D50006946039700941D48FDF78AFF1E4801905D
:108D60006946009502941948FDF782FFE0020090E1
:108D70006946019702951548FDF77AFF174869463D
:108D800091C1694611480397FDF772FF91200002D7
:108D9000694691C10520694600070397FDF768FF02
:108DA00069460A48019700960294FDF761FF002288
:108DB00001210520FEF7B4FA0520FEF7A5FA07B059
:108DC000F0BD00000010024001020000000400504D
:108DD00008300000000011100000211008320000CF
:108DE00010B50F4C0D482060FF200530606000205A
:108DF000A060E06020616061E061012120624902C1
:108E00006062A161A0620720E0622046FEF7D5FE05
:108E10002068016840221143016010BD003001400C
:108E2000A016002010B58AB000240494059406947E
:108E3000079408940121184809940094019402941D
:108E4000890703940160092184604160046113492A
:108E50004461C160FEF77CFF01200003049004A977
:108E60000D48FEF7A3FF0C48FFF792F8089408A9F5
:108E700009480994FEF740FF6020009008480190DF
:108E800002940822694603940348FFF71DF802483C
:108E9000FEF7F4FF0AB010BDF8160020930400009E
:108EA0005702000000B585B014216846FCF77FF931
:108EB0000E480D490160E1214902416000218160B5
:108EC000C160016181610C22C16142610162302196
:108ED00041620121090381634900C163FFF7EEF993
:108EE00001F020FC05B000BD00380140381700201B
:108EF00070470000F0B585B00A2002F061FC7D20CB
:108F0000400102F077FCFC4C0025A570FB48206670
:108F1000A07C2E460C2801D30B20A07460790A286F
:108F200001D90A206071F648E570F64F0078387173
:108F3000F549A079097840000843E17D890008439C
:108F4000F871E06BF870010A3972401CE0636079D7
:108F5000B87442003846ED491330FCF70FF96079D8
:108F6000EA4982004000C01962311330121DFCF73B
:108F700005F96079062142004843C019E4491730D9
:108F8000921CFCF7FBF83020205E002803D0E1495A
:108F9000098A081820866079D749C0002031C21993
:108FA0000B7C53764B7C937606227A72DA4A1D301C
:108FB0001278BA72E28C3A73D24A0B7A133A13756A
:108FC000497A51750022CF4902F0E4FC6079002112
:108FD000C0001D3002F0F0FCD048FEF72FF960858C
:108FE00009E0CE48FEF72AF980B26085218FFF396B
:108FF0002D39884208DB81B2208F8142F1D30122D2
:10900000920380188142ECD8022002F029FCBD486E
:10901000C571E574E573012060742574BF48FEF7DF
:109020000DF9A0850746E5706079FCF749FBBC4A5D
:10903000BC4BFCF729FA01F00DFE0022BA4BFCF7FD
:1090400071F9FCF783FB0006C10CC81980B201213D
:10905000C903E085884201D3401AE085B348E06443
:109060002079401C2071AD48FEF7E8F86085A748DC
:10907000A14F7E3840370190C0E1A848FEF7DEF8E6
:1090800060850BE0A548FEF7D9F880B26085E18DD8
:10909000884203D3A64A8918884207D300210F20AB
:1090A00002F00EFBA34920640842EBD0206C411C67
:1090B0001FD040047ED58122D20100210F2002F072
:1090C0003EFC0021102002F0FBFA41068F48490EB9
:1090D00000229638E16502F029FB002002F08AFBAD
:1090E000002002F03CFB89489638417A0729C3D119
:1090F00001E001F033FC02228F49401DFCF762F8C9
:109100000028B9D102F0A9FCE167A06702F092FC47
:10911000794B803303C3E0787C49401CE0709D3973
:109120000B7A68460370497A417000880390218D5C
:1091300088427DD1734981488C31C98E0180714844
:109140006D498C30008F88847448FEF777F860850D
:1091500002F0C8F968487D22803001684068D20476
:109160000023891858410206080A104341084900A3
:1091700000900A0E080260498031CA608860614828
:10918000E36F0A30A26F02F03DFC607981005D4818
:1091900008185949163080310CC902F033FC564882
:1091A0008030C36882685748123002F02BFC0821D7
:1091B000544800E015E14172B430C07C0009A0754C
:1091C00014D0524802225C499138FBF7FBFF00287B
:1091D0000CD101204B49E074C871E06DCA311638DA
:1091E000C2B24A4822759E30FBF7C8FF6079002260
:1091F000800044491C3002F0CDFB607900218000E2
:109200001C3002F0D9FB009802F0D3FA012002F0E2
:1092100027FB607302214A48FDF7E6FD002823D0B2
:1092200000213948017037498C31488E009000E0A8
:109230008AE03881888E7881FF31844621310A683E
:10924000A06C824201D0761CF6B2E06408602F491F
:1092500020659639C97C0907090F032900D061757B
:10926000E16D1C2902D016E00121DAE72549224AE6
:109270008C31C98F5186264A019B143A1B889382F0
:10928000884207DD002805DD002903D0207E401C30
:10929000207600E0257625710120E0730099B981E0
:1092A0006146F9812074A08C2649FF30C33080B21A
:1092B000A08488420CD949424018A0841F487D22CE
:1092C0000188D200491C89B20180914200D30580F7
:1092D0001A487D210088C9004843A18C4018606568
:1092E00000F060FC607B002805D100210F2002F017
:1092F000E7F90006F9D58AE0700000203F420F0030
:109300001401002034120020480100207E130020A8
:1093100034150020000E00202401002070160020CB
:10932000B81E85EB51B8CE3F00000840A086010072
:10933000983A000000D02724380100204401002082
:1093400000040050E7030000FCF700FF714A03210E
:10935000115471494A8E3A81898E7981E16D224694
:109360001C2905D16D4B4100CB1801990988598002
:1093700080006849684B6039009041189B8F0B80D2
:109380006449303941184B68906C834201D0761C97
:10939000F6B24860604800998C3808186049163069
:1093A0000CC902F02FFBA16C206E814208DA594AE9
:1093B0000098603A1058012802D121660398029063
:1093C0005448009A6038825820468A4216DD012AA5
:1093D00014DD002912DD0399018502210170A573B6
:1093E0000CE0504A00210F2002F0A9FA6079E178E0
:1093F000401C814202D0002002F0B1F9618DE08D65
:10940000814200D239E6484A80188142FAD8E07B8E
:10941000012801D00220E07302F064F8414A0021E3
:109420000F2002F08CFA2079002818D03F490988D3
:109430008A008A18824201D201222270002000F0A4
:10944000EFF8E07C002839D032490C310B78A37258
:10945000487860728A782272022B17D02EE0E16C75
:10946000226E323920468A420EDAC1792F4A491CCF
:10947000C9B2C171128852008A42E2D202990185B2
:1094800002210170A573DCE7E571DAE710280CD042
:10949000C82813D2264BC91C1818FBF76FFE03F01F
:1094A0001FF9642001F03AFC23E6224F386840009F
:1094B000000E03D1C878FCF7E8F83860022E04D813
:1094C000E07A411CE172032800D9E572002023787C
:1094D000A27B657910E00F4E0E4F4100923E7A3F1D
:1094E000765A7F5ABE4205D00B4F02230022012636
:1094F000A6377E52401CC0B2A842ECD32370A273A0
:1095000000F0E4FA074A002180320F2002F017FA37
:1095100005B0F0BD10140020C0120020341500204A
:10952000F000002000D02724983A000024010020F9
:10953000C00D00203C010020F8B52E4C0546E06E21
:109540002D4A281A411E2067914215D21A21615EC8
:10955000081AFCF7A1F8294A294BFBF795FF0646A4
:1095600034200F46205EFCF797F832463B46FBF767
:10957000D9FEFCF7C7F8A086002060761D481C23A2
:10958000C35EC28C1F48008884461F4806881DE0C1
:109590006046484380181D4F80B23880302778439A
:1095A0006427643078431A4F6066C01985420BD235
:1095B000C8B2184934220880606EA25E411BC918E7
:1095C0008918A166E066F8BD491C6176617EB142EA
:1095D000DED33020424310486421101848430F491D
:1095E0004118E16660663421401B615EC018401876
:1095F000A066F8BD70000020CF0700009A999999E5
:109600009999B93F32010020240100204601002031
:1096100078ECFFFF3001002074270000C0BDF0FF90
:10962000FEB5294D2988491C8FB228492F800E8804
:10963000FCF732F8264A274BFBF726FF01910090F2
:1096400025483146FBF754FD244C618F4218B74240
:1096500006D3002028802248019E1018009D02E0B9
:109660001046019E009DFCF72BF833462A46FBF777
:1096700059FEFCF76BF8E086012580B2ED03A842A5
:1096800001D3401BE086E08BFCF71AF8154A164B15
:10969000FBF762FF0646E08E0F460090FCF710F8DD
:1096A00032463B46FBF73EFEFCF750F880B220877F
:1096B000A84201D3401B20870C49009809684861E3
:1096C00000986087FEBD00003001002024010020CA
:1096D0001904560E2D624040E17A0000700000200F
:1096E0001F050000F853E3A59B843E407016002040
:1096F00070470000F8B531492F48086002F094FA2D
:109700002F4800F0A3F92F4CE0822D48801C00F078
:109710009DF920832A48001D00F098F960832B48AA
:1097200029494180014640310979294F0906090E2E
:10973000617006D1C7800121C1870A2141870021BC
:109740008187244AC18E1170C18F2171818F61710F
:10975000817AA1708588052165626181C68830465D
:10976000FBF7C6FCA08101462846FBF7C1FC880038
:10977000081885B2164825816843FBF7A1FF164AF1
:10978000164BFBF7E9FEFBF7E1FFE081658231460E
:109790003846FBF7ADFC20820146C820FBF7A8FC49
:1097A000E0830120A083FCF7E9FCA082E2890C4958
:1097B0000C48FDF747FDF8BD51A7000868000020E0
:1097C000004F00081401002032020000C00D0020EC
:1097D000E803000018000020F853E3A59B843E40F6
:1097E000FF7F000070160020F8B5754C0027754EFD
:1097F0002771012030807449C8200880207B401CDC
:109800002073C00706D0E08C411EE184022801D2FB
:10981000C820E0840120C043FFF702FF0A2001F0C6
:10982000CFFF7D20400101F0E5FF02216748FDF7F1
:10983000DBFA00283FD00020654980000978664D9A
:1098400049000843634909780843A87210206872E8
:109850006248C1887D20C000FBF74AFC68736048FD
:109860005E490078A87328460B308A780270C97860
:1098700041705A49421C20310B7ED370497E1171D0
:109880005649D01C22310B7E5371497E9171534948
:1098900040310A7C0271497C41710022294617201F
:1098A00002F078F80021172002F086F8022001F07B
:1098B000D7FF4C4D03E00120BEE7FEF761FF00211A
:1098C0000F2001F0FDFE28422064F6D0206C411CE0
:1098D00073D040046FD58122D20100210F2002F005
:1098E0002EF80021102001F0EBFE41063A48490E07
:1098F0000022B430E16501F019FF374DB435687AC4
:10990000112858D102223849681DFBF75BFC00285A
:1099100051D1E81F027A69460A70407A4870A97AE4
:109920003180C820FBF7E4FB2749304E0880287BB4
:10993000E08428462838C08E3080294620482839BF
:10994000098F81842A48FDF779FC6085A08C29491C
:10995000FF30C33080B2A08488420BD949424018FE
:10996000A08430882349401C80B20B31308088426B
:1099700000D3378030887D21C9004843A18C40182E
:10998000606500F00FF9684600882085A87C1249C0
:109990006071C731420008460D468330FBF7EEFB8D
:1099A0006079294642001448FBF7E8FBE08CFF2869
:1099B00001D001202070F8BDFFE700F0CFFF0000CC
:1099C000700000202401002032010020000400501B
:1099D000180100201901002034120020C00D0020C1
:1099E0001800002000D02724380100204401002066
:1099F00070160020E70300009613002070B586B0B3
:109A000014216846FBF7D3FB01250F4EED0300221E
:109A100029463046FDF7F5F9012000240190029413
:109A20006946009503943046FDF722F90320019022
:109A300002946946009503943046FDF719F9022017
:109A400001F06CF906B070BD00040050008870474A
:109A500070470000F8B5044600206A461080194D92
:109A600055222A70AA226A700322AA70661DEE701F
:109A70002A716971144A49008918AC712246E81D9F
:109A8000FBF77CFB002007E029186A4689781288DA
:109A900089186A461180401CB042F5DB611DA81C84
:109AA000FCF7A0F801466846018029190078C871C2
:109AB00068464078087221460931024800F044FCAB
:109AC000F8BD0000AE150020C00D002070B52E4C72
:109AD0000C202E4DA07069792D4AC8001730E07017
:109AE00020460C3812880282A88FA071000AE0710B
:109AF00028482B460078207227481A46C0796072A1
:109B000020460C381B8EC3822448203200782073F4
:109B1000E88C60730020A073E073481C207420461A
:109B20000C38137A4377527A82774A0001463E31E5
:109B30001F30FBF723FB68792146820040000019A3
:109B400094311330121DFBF719FB6879062142008E
:109B50004843001912491730921CFBF70FFB687934
:109B6000C100A01C1731FCF73DF868846879C1007A
:109B700028460A192230037853764078907620469A
:109B80001B3100F0C3FD70BD4C130020700000209D
:109B9000380100201401002034120020240100208C
:109BA00034150020FEB5FFF7C7FC2548FDF746FB3E
:109BB000244C86B2668560790A21081AC000FBF73A
:109BC0006BFD07460191A06EFBF77AFD1E4A1F4B05
:109BD000FBF7C2FC00900D463046FBF771FD2B46AB
:109BE000009AFBF79FFB3A46019BFBF79BFBFBF7B9
:109BF000ADFD85B2E586E08BFBF762FD124A134BA3
:109C0000FBF7AAFC06460F462846FBF759FD3246ED
:109C10003B46FBF787FBFBF799FD81B20120C003B0
:109C20002187814201D3091A2187854201D3281A4D
:109C3000E0860349E08E096848616087FEBD000048
:109C40007016002070000020F853E3A59B843E406E
:109C5000034A1168382389B2994301431160704760
:109C60000030014010B5FDF7D9F810BD10B59AB01D
:109C700034216846FBF79BFA14210DA8FBF797FAED
:109C80001C2112A8FBF793FA1B4801680324E40285
:109C9000A143C21489180160FDF74EFB1748016902
:109CA000A143016106200090FF20013002900120B5
:109CB0000390102004900220099040040B900001B2
:109CC00000240C900A946846FDF764FD0F200D9067
:109CD00003200E900F941094012111940DA8FDF70C
:109CE0002FFC81201290032080041890149412A855
:109CF000FDF774FB1AB010BD007000404010024028
:109D000010480168821511430160C1680E4A114074
:109D1000C16001680D4A114001608168490849002D
:109D2000816001680122920491430160C168FD22B3
:109D300012049143C1600021016106490448886012
:109D400070470000001002400C40FF88F6FFF6FE4E
:109D50000050000800ED00E070B5026801239B0789
:109D6000114C124D984203D0A04201D0A84203D119
:109D70007026B2434E683243984203D0A04201D0CD
:109D8000A84204D103231B029A43CB681A438023C1
:109D90009A430B691A4302608A68C2620968816249
:109DA0000121416170BD0000000801400014014024
:109DB00010B5CB06DB0E0121046A99408C43046286
:109DC000016A9A401143016210BD30B58468FF25D5
:109DD0002D021B021343AC430B432343836030BD6E
:109DE000826870239A430A4307210A4382607047BE
:109DF00030B5026A520852000262026A45688369FD
:109E00007024A3439C080B68A40023430224A243AC
:109E10008C6845601443836149684163046230BDC6
:109E200030B5026A10239A430262036A4568826968
:109E300073242402A2430C68240214432022934377
:109E40008A68456012011A4384614968816302622D
:109E500030BD30B5026AFF2301339A430262026AC1
:109E60004568C3697024A3439C080B68A40023437E
:109E700001246402A2438C68456024021443C36138
:109E80004968C163046230BD30B5026A01231B0317
:109E90009A430262036A4568C26973242402A2439A
:109EA0000C68240214430122520393438A684560DC
:109EB00012031A43C46149680164026230BD30B5BF
:109EC000036A046A6408640004628469F025AC4390
:109ED000120122430A24A3430B438261036230BD73
:109EE00030B5036A1024A34303628469036A0F2513
:109EF0002D031203AC432243A024A34309011943B9
:109F00008261016230BD0000F8B5102405252D07DF
:109F1000AC62AF20800000F008FFAC6101F0E4FB10
:109F20002D4C2E4F2E4E60670EE001F0DDFB60677A
:109F3000FEF726FC606C411C6164142804D929A03A
:109F400000F08EFC2B48C760606FB042EDD1002658
:109F5000666420780127FF03030000F0BAFC0403C5
:109F60000B182C2E012239462846FCF74AFFFFF732
:109F70003BFC06E0012239462846FCF742FFFBF78E
:109F800061FE002239462846FCF73BFF15E0A07B26
:109F90000122401CA07339462846FCF732FFFCF72B
:109FA00009F9002239462846FCF72BFFA07B05283B
:109FB00003D9267001E0FEF79DFF02210E48FCF751
:109FC00013FF002805D000200C49087001F072FA38
:109FD000F8BD0120F8E70000700000200400FA0539
:109FE0003001CADE4457204944204552524F522E78
:109FF0000D0A000000ED00E00004005048010020C0
:10A0000010B5818CC90707D001684A6801235B0439
:10A010009A43836A1A434A60818C890707D501688D
:10A020004A6801231B049A43C36A1A434A60818C1D
:10A03000490707D501684A6801239B049A43036BCB
:10A040001A434A60818C090707D501684A680123D1
:10A05000DB039A43436B1A434A60818CC90607D5D8
:10A060000268916801231B039943836B1943916034
:10A07000818C890607D501688A6801235B039A43AE
:10A08000C36B1A438A60818C490612D503685A68EB
:10A0900001210905046C8A4322435A60026C8A42FA
:10A0A00007D10268516803235B059943436C194348
:10A0B0005160818C090607D501684A680123DB04D9
:10A0C000806C9A4302434A6010BD0000F8B5044614
:10A0D000002680300660FCF79BFE0546206800687D
:10A0E000124F000709D501212B46002249052046C1
:10A0F000009700F0A1FA00280DD120680068400701
:10A100000BD501212B46002289052046009700F03F
:10A1100093FA002801D00320F8BD2020A067E06753
:10A120002666603426750020F8BD0000FFFFFF01A1
:10A13000F8B5154CC826E078002823D160790028AE
:10A1400020D101206071114D686B0027002818D0C4
:10A15000686BC821081A0FE00D48E168405C61692E
:10A160008847E068401CE060E068C82800DBE760E2
:10A17000696BC820401A761EE168814201D0002E2A
:10A18000EADC6771F8BD00005400002000000240C6
:10A19000F80C002070B5224CE07800283FD12079DF
:10A1A00000283CD1012020711E4EF16900250906CE
:10A1B000002933DA2156625791420AD1F0694006EC
:10A1C0002CD5A079002829D0A5712089401C208198
:10A1D00024E0A179002903D1A0710A2000F0A5FD97
:10A1E00000202056CC2148430F49421820691218FC
:10A1F0001279B262401C00222061A256CC235A433D
:10A20000895881420ADC25612078401C2070207822
:10A210000E2800D12570A078401CA070257170BD5B
:10A220005400002000380140D001002010B5806AA1
:10A230000022014640314A834A82FDF72DFF10BDBE
:10A2400070B5846AA06FE56F2168896800260906E9
:10A25000002906DA212804D152200653204600F0B6
:10A260006BF820688068400606D5222D04D15A205C
:10A270000653204600F047F820468030016810223F
:10A28000114301602046FDF707FF70BD10B5014680
:10A290000968806A096889061CD400225A210A527A
:10A2A00001680A68FF2301339A430A6001688A68DB
:10A2B000520852008A6001688A6840239A438A6083
:10A2C0002021C167016E012904D101680A681023A9
:10A2D0009A430A60016E012902D0FEF7BFF810BD53
:10A2E0005821095AFDF7D6FE10BD10B5806A016EDF
:10A2F000012902D0FEF7B3F810BD5821095A4908C8
:10A30000FDF7C8FE10BD01680A68FF2321339A4398
:10A310000A6001688A68520852008A60016E012949
:10A3200004D101680A6810239A430A602021C1679A
:10A33000002101664166704701680A68C0239A439C
:10A340000A6020218167704770B5164CE278002AB8
:10A350000CD12279002A09D10122E2700025C829F6
:10A3600003DC0222A256002A01DCE57070BD012345
:10A37000E356CC2253430C4AD1500123E356CC265A
:10A3800073439B180A460146181DFAF7F7FE6078DA
:10A39000401C607060780E2800D16570A078401E67
:10A3A000A070E2E754000020D0010020F8B5044678
:10A3B000016880682369E6691843636900253343AF
:10A3C0001843724A0B68724E334003430B60216896
:10A3D000486803231B039843E368184348602168D7
:10A3E000A069914201D0236A18438B680B2636027C
:10A3F000B34303438B606749236867488B420CD1A2
:10A40000C0688007800F06D0012839D0022835D0D7
:10A41000032821D11EE001271FE060498B420AD1A9
:10A42000C0680C21084027D0042829D0082825D04E
:10A430000C2811D10EE093420ED1C1680320800296
:10A44000014019D001208002091A19D0091A15D02B
:10A45000814201D1082700E010274F495048403978
:10A460008600934232D1002F0CD0022F0DD0042F42
:10A4700010D0082F7FD126E00027EEE70227ECE777
:10A480000427EAE7FDF72AF906E00968C90605D4BA
:10A49000304603E0FDF742F9002872D062685100AF
:10A4A0005118814267D81103814264D3010E06021C
:10A4B0005008002330185941FAF730FE03210902F1
:10A4C000411A384A55E00120C003E7E70122E36959
:10A4D000D20393422BD13B0000F0FBF90906090C93
:10A4E0004D114D4D4D274D00FDF7F8F809E0FDF7F2
:10A4F00005F906E00968C90605D4304603E0FDF712
:10A500000DF900283DD0616840004A088018FAF72C
:10A51000EFFD80B20146244A103991422BD8511CDC
:10A5200001400007400F084329E01046EBE73B00DD
:10A5300000F0CFF90906090C211221212123210065
:10A54000FDF7CCF80AE0FDF7D9F807E00968C9067D
:10A5500006D4304604E00EE0FDF7E0F8002810D005
:10A5600061684A081018FAF7C3FD80B201460E4A26
:10A570001039914203D9012503E01046F0E7216824
:10A58000C86000206066A0662846F8BD004800400C
:10A59000F369FFEF003801404010024000440040E2
:10A5A00000093D00FFFC0F00EFFF0000F8B5044676
:10A5B0004165403000262746028380373E602220D6
:10A5C000E0672546206F603500281CD01749C1621E
:10A5D000216F17480863216F16484863206F866310
:10A5E000236F606D9C461346216802466046243105
:10A5F000FCF766FA002806D0102038602E7520205F
:10A60000A0670120F8BD2E7520680168FF22013285
:10A610001143016020688168012211438160206834
:10A6200081684022114381600020F8BD8DA200089E
:10A63000EBA2000841A20008FFB581B005460F4615
:10A64000044660350A9E39E0701C37D0FCF7E0FB09
:10A650000499401AB04222D8002E20D02068016808
:10A6600049072BD5C069C043000527D401202168C4
:10A67000C002086220680168FF22A1329143016094
:10A68000206881684908490081602020A067E06750
:10A690008034206000202875032005B0F0BD2068BC
:10A6A0000168FF22A1329143016020688168490856
:10A6B000490081602020A067E067EBE72068C1695E
:10A6C0003846884305D0002103988142BCD0002041
:10A6D000E3E70121F8E7000010B5044910200968FC
:10A6E00008620248FDF7DAFC10BD000038170020B0
:10A6F00001B501231A4669460248FDF7B1FE02483A
:10A70000C06908BD381700200038014070B50D46FB
:10A710000646002403E0305DFFF7EAFF641CAC420C
:10A72000F9DB70BD01490D2088707047540000208E
:10A7300010B5FEF79DFAFEF7B5FBC82202490348A3
:10A74000FDF75CFE10BD0000F80C0020381700205B
:10A75000F8B53E4C002321783D4A1D46082910D00B
:10A76000072947D0062950D0052952D0042953D0B3
:10A77000032954D0002956D0012958D002295AD093
:10A780005BE0A17800264A1F04E0314FBF5DFB1853
:10A790009BB2761C9642F8DB667927799A19511894
:10A7A000E3786278C9188918C9194018C0430006AF
:10A7B000000E1AD1012E14D0022E16D1254824499C
:10A7C000C018FAF7DBFC01F08BFF642000F0A6FA5A
:10A7D000BFF34F8F21492048C860BFF34F8F00BFA0
:10A7E000FDE759081046FFF735F92570E570A570AB
:10A7F000A571F8BDA1795054491CC8B2A071A178C7
:10A80000491F8842F5D1082001E0607007202070C0
:10A81000F8BDE0700620FAE760710520F7E7A07048
:10A82000E5700420F3E7552807D10120EFE7AA28B7
:10A8300003D10220EBE7032803D02570E570A57053
:10A84000F8BD032020702071F8BD00000B0100202E
:10A850004A150020C00D00200400FA0500ED00E0BC
:10A8600010B5024A024900F0E5F910BD1DBA000812
:10A87000600100202021020C01D010211046020AA4
:10A8800001D010460839020901D01046091F82087C
:10A8900001D01046891E420801D0881E7047081A50
:10A8A0007047F8B5040C8BB2264682B25E430D0C9D
:10A8B0001046370C5843360480190021794116465A
:10A8C0006E43370C36048019794126466E43891948
:10A8D000F8BD30B47446641E2578641CAB4200D2C7
:10A8E0001D46635D5B00E31830BC18474900CA028F
:10A8F0000243100000D004204A0D01D00122104371
:10A90000044A490D914201D102210843012800D196
:10A9100005207047FF0700008307FF22DB0E9A40E7
:10A920008907090E9940002808DB830809489B0025
:10A930001B18186890430843186070470007000F01
:10A940000838830804489B001B18D86990430843C3
:10A95000D861704700E400E000ED00E0BFF34F8FE6
:10A9600004490348C860BFF34F8F00BFFDE70000F4
:10A970000400FA0500ED00E0F8B504464F1EC800DB
:10A980000838211815461E46086849683A460623C5
:10A990009A4310D02A463346FAF776FD3A46D2005B
:10A9A000083AA3181A687F1E5B68FAF7BBFC0622F8
:10A9B0003B469343EED1022F23D0042F11D0062F14
:10A9C0002FD12A463346FAF75FFDE36AA26AFAF707
:10A9D000A9FC2A463346FAF757FD636A226AFAF75A
:10A9E000A1FC2A463346FAF74FFDE369A269FAF75C
:10A9F00099FC2A463346FAF747FD63692269FAF75C
:10AA000091FC2A463346FAF73FFDE368A268FAF75D
:10AA100089FC2A463346FAF737FD63682268FAF75D
:10AA200081FCF8BD002210B5134610460149FAF723
:10AA300093FD10BD0000F03F10B5FAF773FC10BD98
:10AA4000002210B5134610461146FAF785FD10BDD9
:10AA500010B50721024A00200907FAF7F5FD10BDDD
:10AA600001030000034A10B500201107FAF7ECFDBE
:10AA700010BD000001FDFFFF02E008C8121F08C161
:10AA8000002AFAD170477047002001E001C1121F6F
:10AA9000002AFBD1704700000149086070470000A0
:10AAA0006401002008B50021684601706B46012250
:10AAB00002212C2000F052FF0221684601706B46F3
:10AAC00001222C2000F04AFF08BD000038B50446E2
:10AAD0006D20694608706B46012207492E2000F060
:10AAE0003DFF0649002C01D0054A00E0054A2E2012
:10AAF00000F01AFF38BD000006080000061800002C
:10AB0000070600000716000038B504466B4602220F
:10AB10000021362000F0EEFDB3212300FFF7D9FE1F
:10AB20000E0F08153A3A3A3A1C273A3A2F34483A67
:10AB300000216846017040784108490014E06946E8
:10AB4000087880088000401C04E069460878800886
:10AB50008000801C08701DE0684602780A40483278
:10AB600002704178802001436846417012E06846D7
:10AB700002780A40027040784106490EF4E76946BF
:10AB800048780221084303E069464878FD210840DF
:10AB9000694648706B4601220021362000F0DEFE37
:10ABA000012200AB11463620013300F0D7FE38BD3C
:10ABB00069460878CF21084069462030CAE708B5C1
:10ABC000032168464170012101706B460222002179
:10ABD000362000F0C3FE0122D20306212D2000F012
:10ABE000A3FE012000F09AF80120FFF78DFF08BDB9
:10ABF00008B5020A69464A7008706B4602220421B1
:10AC00002D2000F0ABFE0320694608706B46012240
:10AC100006212D2000F0A2FE0020694608706B4638
:10AC2000012206212D2000F099FE0A212D2000F09E
:10AC300047FD08BDF8B516460F460446002503E05B
:10AC40003946B047641C6D1C20780028F8D128468E
:10AC5000F8BD0000F8B54A002B4B520DD6182B4A10
:10AC60000C460546142E2BDA002E12DA284BFAF782
:10AC700059FB00221346FAF7AFFD40D2002C03DA4D
:10AC80000124E40700253AE02046284337D0214C30
:10AC900014E0214F0B46F7403B402B4331D01C4B77
:10ACA000FAF740FB00221346FAF796FD27D2002C54
:10ACB00003DD01200005F0400419BC4300251EE01F
:10ACC000332E1EDC33460027143BFF43DF4038425F
:10ACD00017D00F4BFAF7D0FB00221346FAF77CFD92
:10ACE0000DD2002C0ADD142E0CD03420811B012043
:10ACF00088404019A84200D2641C0546BD43214645
:10AD00002846F8BD641CF9E701FCFFFF9C7500882C
:10AD10003CE4377E0000F03FFFFF0F007D2110B5BF
:10AD2000C900484300F001F810BD002140E000BF19
:10AD300000BF00BF00BF00BF00BF00BF00BF00BF1B
:10AD400000BF00BF00BF00BF00BF00BF00BF00BF0B
:10AD500000BF00BF00BF00BF00BF00BF00BF00BFFB
:10AD600000BF00BF00BF00BF00BF00BF00BF00BFEB
:10AD700000BF00BF00BF00BF00BF00BF00BF00BFDB
:10AD800000BF00BF00BF00BF00BF00BF00BF00BFCB
:10AD900000BF00BF00BF00BF00BF00BF00BF00BFBB
:10ADA00000BF00BF00BF00BF00BF00BF00BF491C05
:10ADB0008142BCD37047FFB581B01E460F460400E8
:10ADC00026D00B9903980143A06A39438268072073
:10ADD0009047002818DB0A99A06A31438268062050
:10ADE0009047002810DB25462035A979032F01D98B
:10ADF00008200143032E01D904200143A06A826880
:10AE000009209047002806DA0120C04305B0F0BDB4
:10AE10000020C043FAE7384600F000F920603046D1
:10AE200000F0FCF860600A9868700398A870EF70F2
:10AE30002E710B9868710020E8E70000F7B5044612
:10AE4000002090B000900190002C05D06A460621A9
:10AE500001F080FC062803DA0020C04313B0F0BDE7
:10AE60006846407801026846007800040918684680
:10AE700080780818FAF724FC0546684603910079A3
:10AE800001026846C078000409186846407908182D
:10AE9000FAF716FC032206460F4692075C4BFAF7B8
:10AEA0009BFC07D200225B4B30463946FAF7DEFAAC
:10AEB00006460F4603229207554B28460399FAF798
:10AEC0008BFC07D20022534B28460399FAF7CEFA9F
:10AED000054603912068FAF7F3FB02460B4630461D
:10AEE0003946FAF739FB07460A200791205EFAF740
:10AEF000D3FB3A46079BFAF7C7FA064608200991A2
:10AF0000205EFAF7B7FB0021C943FAF7FFF9FAF719
:10AF10003BFC3246099BFAF705FA069108906068F7
:10AF2000FAF7CEFB02460B4628460399FAF714FBC4
:10AF300005461A200E46205EFAF7AEFB2A46334637
:10AF4000FAF7A2FA0C9009911620205EFAF7A4FBFA
:10AF5000099B0C9AFAF7E6F905910A902A463346BE
:10AF600038460799FAF790FA059B0A9AFAF78CFA8D
:10AF700005910A901420205EFAF78EFB3A46079B53
:10AF8000FAF782FA07461C200791205EFAF784FB45
:10AF90002A463346FAF778FA0E900B911820205E75
:10AFA000FAF77AFB0B9B0E9AFAF7BCF92A4633465E
:10AFB000FAF76AFA0B910E902069FAF76DFB0B9B7A
:10AFC0000E9AFAF7AFF92A463346FAF75DFA0546C4
:10AFD0000E46E068FAF760FB2A463346FAF7A2F914
:10AFE0003A46079BFAF79EF9059B0A9AFAF79AF9EF
:10AFF00001229207084BFAF747FA02460B46129CC9
:10B000000898069903C411980CC0002026E7000098
:10B01000FFFF5F4100007041E17A843F00B50121EC
:10B02000C9040300FFF755FC081A05080B0E11149C
:10B03000171A0320C00400BD0720C00400BD0F2064
:10B04000C00400BD1F20400300BD3F20400300BDE1
:10B050007F20400300BDFF20400300BD084600BD27
:10B06000FEB5264F0D4604000FD0002D0DD026460C
:10B0700000202036B071F07129680D208847002823
:10B0800001DA7800FEBD102801D03846FEBDA56269
:10B09000E968002901D028208847204600F030F8D0
:10B0A0000028F3DBA06AA52182680E209047A06AE1
:10B0B000962182680F209047A06A02218268622050
:10B0C0009047A06A002182680E209047A06A002164
:10B0D00082680F20904771793020019100900623FB
:10B0E000202201212046FFF766FE0028CEDB204605
:10B0F00000F0AEF80028C9DB0020FEBDFFFFFFFF17
:10B1000010B586B0044614216846FAF750F8002CB2
:10B110007ED0A06A122143686A4610209847122800
:10B1200077D1684600780122010168464078120311
:10B130000009081843492081884201DD801A2081D6
:10B140006846837840780007000D181860818842AF
:10B1500001DD801A6081684600790122010168469C
:10B16000C0781205000309186846407900090818DC
:10B170003549E060884201DD801AE0606846407928
:10B180000007030B6846807900021B186846C079E7
:10B1900018182061884201DD801A20616846417AD2
:10B1A000007A0002081802B2284801210904A2828C
:10B1B000824201DD521AA2826A46D37A927A120240
:10B1C0009A1812B2E282824201DD521AE2826A4683
:10B1D000537B127B12029A1812B22283824201DD43
:10B1E000521A22836A46D37B927B12029A1812B2B9
:10B1F0006283824201DD521A62836A46537C127C6A
:10B2000012029A1812B2A283824204DD501A01E09F
:10B210000BE008E0A083A06A016828208847002886
:10B2200006DA0120C04306B010BD0020C043FAE793
:10B23000C011C0072034002800D080206071002099
:10B24000F1E70000FF070000FFFF0700FF7F00009D
:10B2500010B5040009D0A06A072182680820904731
:10B26000002805DA0120C04310BD0020C04310BDF6
:10B27000072020342070002010BD0000FEB50446D9
:10B280000020019000906079734940000E5A617867
:10B290002578491E7148CFB20163042D77D0072D60
:10B2A00075D000210291217801736C49E379012264
:10B2B00092058969002B6CD0914381616748217A9E
:10B2C0004173217A82698907890B0A4382610021CF
:10B2D000042000F034FB324661492E2000F024FBAC
:10B2E0003846FFF7F3FB5F4E0522705D8100401882
:10B2F0005D49431807212B2000F030FB5B49029881
:10B3000001220B180B21282000F028FB705D584902
:10B3100080000A580C21282000F011FBE0795549E3
:10B3200080004018A1794900425A0221272000F0EC
:10B33000FBFA51487E00825B0421272000F0F4FADA
:10B34000E079002829D0A07804282CD0282069464C
:10B35000087220220621272000F0E6FA02AB012223
:10B360002621272000F0FAFA444938014018E178F4
:10B37000890042580821272000F0E1FAA17A601CD8
:10B38000627A0902114313D016E000E001E00121C6
:10B3900088E71143F608816190E76422062127209F
:10B3A00000F0C2FAE0E71020694608720246D1E7D1
:10B3B00033490172090A4172417A007A0A02024352
:10B3C0002021272000F0B0FA2E4F0C2123203A68CC
:10B3D00000F0B5FAF01982880421232000F0A4FAC5
:10B3E000A07900280BD0E0792749012243180021D9
:10B3F000212000F0B3FA03200190012000902A07D9
:10B40000120F10010243607800218007000B0243F5
:10B410000198000502430098400402432079C006C9
:10B42000400902436079C00602431F2000F087FAFA
:10B43000A07861780123084302040848DB03026115
:10B44000E179490319430A4302610021082000F011
:10B4500076FA0020FEBD000088C800089401002094
:10B460000428000030C8000824000020420000200A
:10B4700038C8000858C8000864C8000868C8000830
:10B480004110000050C800084400002038B50C46A8
:10B4900007498A8B002102432C2000F045FA6846B8
:10B4A00004706B46012206212C2000F057FA38BDAB
:10B4B0009401002010B5FFF7F5FA10BD10B5044651
:10B4C0000421362000F0FCF80121C902002C01D033
:10B4D000084300E0884302460421362000F02FFA9A
:10B4E00010BD000038B540206946087000210E20CC
:10B4F00000F0E6F80446002211460E2000F01FFA84
:10B500006B46012200210D2000F028FA074A002195
:10B510000F2000F014FA00F0EDF9224600210E2071
:10B5200000F00DFA02480021017338BDF8FF27240E
:10B53000B4010020FEB50546042069460870514C50
:10B540000020607521462031206348710873A08374
:10B550006063A06300F0C8F84B4E206002E000F08A
:10B56000C3F82060B042FAD10020FFF7CDFA00F016
:10B57000BBF8464E20603078242801D9243806E0F4
:10B580000621F9F7B5FD0622101A4001084302060C
:10B5900001040A4301020A430243B26070600021C1
:10B5A0001E2000F0CCF900F09FF820606B460122CD
:10B5B0000021242000F0D2F91E20FFF719FB86B2EB
:10B5C000300AA0730420FFF713FB074600F08CF845
:10B5D00020603806000E0DD002206946087101ABCC
:10B5E000012212212D2000F0B9F9A08B01210903BD
:10B5F0000843A08300F078F820600620FFF7F8FAEF
:10B6000060600720FFF7F4FAA060F006C00E207516
:10B6100001D110202075C0B200F0DCF9E80707D096
:10B62000FFF7CDFAA08B0121C9020843A0830AE0ED
:10B630000521362000F02EF8154908400246052164
:10B64000362000F071F90120FFF75EFA0021042096
:10B6500000F036F8A0610021262000F031F8152115
:10B660008903084302460021262000F068F90022E1
:10B670002621362000F058F900F036F8206000202E
:10B68000FEBD0000940100203001CADE1800002039
:10B69000FFFD000038B5094C89B280B26B4602222A
:10B6A00000F028F8002806D1684640780102684674
:10B6B0000078081884B2204638BD0000FFFF000063
:10B6C00038B50024E44389B280B26B46042200F00E
:10B6D00011F8002806D103216846435C2202D418E1
:10B6E000491EFAD5204638BD10B500210846FFF79F
:10B6F000E7FF10BD38B5002909D0402420436C462F
:10B700002070C8B27F2906D8607002200AE069461E
:10B710000870012006E0802420436C466070C80950
:10B72000A0700320694600F0B5FF38BD10B514467F
:10B7300003460A4621461120FFF7DCFF10BD10B575
:10B740000346052200211520FFF7D4FF10BD10B5D8
:10B750000346052200211720FFF7CCFF10BD38B5A6
:10B76000054600206946087000F0C4F8FF24013443
:10B770002246002D01D00322120200210D2000F0EC
:10B78000D3F8002D13D06B46012203210F20FFF7C1
:10B79000B1FF68460078000709D5FFF7A3FE2246EF
:10B7A00000210D2000F0C0F80020C04338BD00206B
:10B7B00038BD10B5024601210A2000F0C0F810BDC6
:10B7C00010B5044600211A20FFF77AFF000D22036E
:10B7D0000005120B024300211A2000F0B0F810BD42
:10B7E00010B5024602492E2000F09EF810BD000060
:10B7F00004180000F8B505466B4601220321042019
:10B80000FFF778FF0126114C3607002D0DD02A4690
:10B8100000210C2000F088F86946087810210843C0
:10B8200069460870A069304307E069460878EF214F
:10B83000084069460870A069B0430B46A061012228
:10B840000321042000F08AF8F8BD000094010020D4
:10B8500010B502460021182000F066F810BD000067
:10B86000F8B50746002568460570B807204C2E46F7
:10B8700000280ADA8020694608706B460122002100
:10B880000D2000F06BF801202073F8076946087856
:10B8900021D006210843694608706B460122002129
:10B8A0000D2000F05BF803210F20FFF7F3FE81214C
:10B8B000C900084219D04020694608706B46012231
:10B8C00000210D2000F04AF80020FFF7F7FD0025C9
:10B8D0002673ED4309E002210843694608706B4670
:10B8E000012200210D2000F039F82846F8BD0000A3
:10B8F000B40100201CB56B46012203210F20FFF785
:10B90000F9FE684600784022C1091040C901400094
:10B91000814208D0012069460871024601AB03212B
:10B920000D2000F01BF81CBD08B56B461A70120AFA
:10B930005A7089B280B2022200F010F808BD38B502
:10B9400000236C46E254120A5B1C042BFADB89B21A
:10B9500080B22346042200F001F838BD38B58024B7
:10B96000002909D0C02528436D462870C8B27F2918
:10B9700007D86870022009E020436946087001205A
:10B9800004E020436870C809A8700320694600F0ED
:10B990002BFF38BD10B51446012312189B029A42A2
:10B9A00002D90020C04310BD0B46821E214609204B
:10B9B000FFF7D4FF002010BD10B5054A89051269B4
:10B9C00001430A4300210820FFF7B9FF002010BD02
:10B9D0009401002038B504466B4601220E212B202D
:10B9E000FFF788FE68460078E10640094001C90E6D
:10B9F0000143684601706B4601220E212B20FFF7A0
:10BA0000ADFF38BD10B5002142541C06120A224376
:10BA10001B0A491C0429F7DB10BD000013B50123E4
:10BA20001A4669460248FCF71BFD00981CBD000041
:10BA3000381700207CB5002425466846FFF77FFEB6
:10BA400004206946220E2D02154322020C5C144389
:10BA5000401EF7D5204629467CBD7CB500242546EE
:10BA60006846FFF774FE04206946220E2D02154336
:10BA700022020C5C1443401EF7D5204629467CBDAB
:10BA8000FBF7D4F9FEF7F2F8FDF706F93F49404815
:10BA9000002522C005608561C5613E490562C1601F
:10BAA0000838FBF755FBFDF7E3F8FDF7FBF9FDF769
:10BAB00097F9FDF7A9F8052401222407D1032046B0
:10BAC000FBF79FF9FDF716FEFCF786FFFAF766F81D
:10BAD000FAF712FAFAF7E0F9FCF744FD0721A0158E
:10BAE000FFF7D4FCFFF7E6FC012211032046FBF729
:10BAF00088F92748C8222849C830FCF77FFCFCF7A2
:10BB000019FF264F264E274C387800280FD1307861
:10BB1000002801D003280AD10121C9022248FBF7DD
:10BB200063F9002803D101210846FBF725FCE078E2
:10BB3000002828D06078002825D0E57072B62078DB
:10BB40000F280AD90120184900038861FEF7DCF9A3
:10BB500001201549000388620CE0012251031248BC
:10BB6000FBF74FF9FEF7D0F90121002249030E48F7
:10BB7000FBF747F962B6FCF703FE208C0028C3D020
:10BB8000401E2084C0E7FCF7FBFDBDE7007C0040C1
:10BB900070160020FFFF0000F80C00205A00002063
:10BBA00085000020140100200004005010B586B06C
:10BBB0001848FBF750FA14216846F9F7F8FA1648C6
:10BBC00000900320019000200290052069460007A4
:10BBD000FBF74EF869461148FBF74AF869461048EA
:10BBE000FBF746F8FCF7A6FE01210846FBF7C4FB6D
:10BBF000FF2401342046FBF797FB0A49086804221A
:10BC0000104308602046FBF79FFBFBF7A5FB06B03F
:10BC100010BD000070160020FFFF0000000400505F
:10BC2000000800500070004010B501229202174930
:10BC30001748FAF7E5F91548164902888A4223D0D1
:10BC4000018004218180FF21F531C1800A21018119
:10BC500000211E224181D24382810122C28181833F
:10BC60004323C38602230387782343878287C287BF
:10BC700002464032118451849184C18391801423FF
:10BC80008382118200F02CFD10BD0000C00D002049
:10BC900000FC0008AA550000F0B51FB496B0844619
:10BCA0000C460246199D18980390490068006300ED
:10BCB000490840080193002A01D0012600E000262F
:10BCC0009E19FE4BF6185B109E422BD36E00039F0D
:10BCD0000296002F00D00127F719F84EF84BBE1935
:10BCE0009E421FD3039E0346F64F334309D03B4683
:10BCF0009C4201D1002A04D0019B002A05D00126D4
:10BD000004E0002039461BB0F0BD00269E19EE4B22
:10BD10009E4207D8039F029E002F00D00127F619EC
:10BD20009E4207D92B4660462146189AFEF784FEAC
:10BD30001BB0F0BD0023002C29DAE44EB04226DA15
:10BD4000E34EB04201DB022321E0DE4EB0421EDBB7
:10BD5000E04E070DBE19142E09DD3427BF1B039ECC
:10BD6000FE400196BE40039FBE420BD00FE0039FF2
:10BD7000002F0CD11427BF1B0646FE400196BE4083
:10BD8000864204D1019BDE07F60F02239B1B0E4661
:10BD9000164318D1002D16DA002C03D0022B01D047
:10BDA000012B06D00220FEF777FEFEF73BFE1BB00C
:10BDB000F0BD0220FEF770FEFEF734FE0122D2072E
:10BDC00051401BB0F0BD039E002E61D1BF4EB0426A
:10BDD00020D1C148844201D1002A08D0B94881420B
:10BDE00009DB002D10DB189829461BB0F0BD0020A0
:10BDF000B4491BB0F0BD002D06DA01222946D20756
:10BE0000189851401BB0F0BDB4497944086849689E
:10BE10001BB0F0BDAB4FB84225D1002D1FDA002971
:10BE200004D0B14212D1002A09D018E0002A72D100
:10BE3000A649E20F0020D20711431BB0F0BD00203D
:10BE4000E20F0146D20711431BB0F0BDB14206DA42
:10BE5000234600203946F9F77FFB1BB0F0BD1046A2
:10BE600021461BB0F0BDB14212DA0126B607B54239
:10BE700003D1234610461946FEE3994EB54207D139
:10BE8000261E05DB1046314600F040FC1BB0F0BD1D
:10BE900067007F081646002A40D100290AD08B4A45
:10BEA000914229D1002C0EDD002D1CDB0020114613
:10BEB0001BB0F0BD022B16D0002C14D0012B12D1D8
:10BEC000002C14DB0FE0002C28DA002D09DB012BFD
:10BED00003D000207D491BB0F0BD002081491BB07C
:10BEE000F0BD012B03D0002001461BB0F0BD0020A7
:10BEF0000121C9071BB0F0BD724A91420ED1002C3E
:10BF000001DA002B17D0022B06D00020C043F9F72E
:10BF1000C3FB1BB0F0BD90E20120F8E7E217521C12
:10BF200094461A4307D000220892664C62465B1E74
:10BF30001A4307D009E00120FEF7AEFDFEF780FDB1
:10BF40001BB0F0BD0022644C0892674A90427DDD30
:10BF5000664B674A98421FDD914202DC002D05DBEB
:10BF60004DE05848814217DB002D48DD0220FEF7E6
:10BF700093FDFEF76DFD05460E460022534B21460C
:10BF80000898F9F781FA084671004908C00FC00700
:10BF9000014328461BB0F0BD914215DA002D2EDA80
:10BFA0000220FEF779FDFEF753FD05460E460022FE
:10BFB000464B21460898F9F767FA72005208C80FF5
:10BFC000C0070243114617E03E4B994223DD002D86
:10BFD00015DD0220FEF760FDFEF73AFD05460E4630
:10BFE00000223A4B21460898F9F74EFA08467100AC
:10BFF0004908C00FC007014328461BB0F0BD02200E
:10C00000FEF74AFDFEF72EFD49004908E20FD20770
:10C0100011431BB0F0BD002230463946F9F726FA2D
:10C02000012205460E46D243F9F70EFB314A324B48
:10C03000F9F722FA2A463346F9F726FA0022284B66
:10C04000F9F71AFA07462A46334600E064E00391FE
:10C0500010461946F9F718FA3A46039BF9F714FA0D
:10C060000746032209915207244B28463146F9F727
:10C070000BFA07910C90224A204B38460999F9F7A0
:10C0800003FA074601911F4A1F4B28463146F9F72C
:10C09000FBF93A46019BF9F7E9F907460B460246D8
:10C0A000099107990C98F9F73DF900250E462846A5
:10C0B000079B0C9AF9F7DAF93A4627E0FFFF1F00D1
:10C0C000FFFF0F000000F03F0000E0FF0000F07FE6
:10C0D0000000404301FCFFFF0000F0BF5A0B0000CE
:10C0E0000000E03F0000F0FF0000E0410000F043EE
:10C0F000FFFFEF3F555555555555D53F4715F73F70
:10C10000FE822B6544DF5DF80BAE543E099BF9F7C8
:10C11000B3F902460B4652E1012500202D05A94244
:10C1200007DA352230463946F9F78EFA06463420CA
:10C13000C0430A151218FE48101803900803FD4961
:10C14000000B01430F46FC49884201DC002003E05C
:10C15000FA49884202DA0120119005E0002011908E
:10C160000398401C7F1B039011980597C200F44868
:10C170000F927844801843680268394630460D9320
:10C180000292F9F773F907910C9030460D9B029AD1
:10C190000599F9F7C7F802460B460020E549F9F77B
:10C1A000DBF909910490079B0C9AF9F76DF912904D
:10C1B00000201090E3480D46784400680E9001215D
:10C1C00078104907084311990D9B890440180121F3
:10C1D000C90447183946029A0E98F9F747F93246CA
:10C1E000059BF9F749F902460B4629461098F9F7DD
:10C1F0004BF9064602913B4629460E9A1098F9F7EC
:10C2000043F9079B0C9AF9F737F93246029BF9F785
:10C210002DF9099B049AF9F737F90591129A0A90BA
:10C220002B4610461946F9F72FF906460246C6482E
:10C230000F460B4606217844FEF79EFB32463B46EE
:10C240000091049010461946F9F71EF9009B049AD4
:10C25000F9F71AF906460F462B461946129A109816
:10C26000F9F760F8059B0A9AF9F70EF932463B4652
:10C27000F9F758F8109A079104902B461046194682
:10C28000F9F702F9B14E0022334609910290F9F70D
:10C2900049F8079B049AF9F745F80020074602463B
:10C2A00033460091F9F7E2F8099B029AF9F7DEF8B4
:10C2B000079B049AF9F7E0F806460D913A4629469D
:10C2C000009B1098F9F7E0F807910C902B46304648
:10C2D000129A0D99F9F7D8F805460E463A46009B92
:10C2E00005990A98F9F7D0F833462A46F9F71AF86B
:10C2F00002460B460746099107990C98F9F712F880
:10C3000000250E462846079B0C9AF9F7AFF83A46E7
:10C31000099BF9F7B1F807460722099152078C4BA0
:10C3200031462846F9F7B0F807910090894A884BC2
:10C3300038460999F9F7A8F807460191864A874BCC
:10C3400031462846F9F7A0F83A46019BF8F7EAFF8C
:10C35000834B7B440F9A9B181A685B68F8F7E2FFDF
:10C36000029009910398F9F797F905910490099BB8
:10C37000029A07990098F8F7D5FF7A4B7B440F9AF9
:10C380009B181A685B6817460393F8F7CBFF059B69
:10C39000049AF8F7C7FF0E462846059B049AF9F75A
:10C3A00065F83A46039BF9F761F8079B009AF9F79D
:10C3B0005DF8099B029AF9F75FF802460B46199956
:10C3C00000200C900F461898F9F75EF8029104903F
:10C3D0003B460C9A19991898F9F748F82A463346BB
:10C3E000F9F752F8029B049AF8F79CFF09910E9016
:10C3F0002A46334639460C98F9F746F806460F4662
:10C40000099B0E9AF8F78EFF574A0D46914220DBA2
:10C410005242AA18024310D132463B46F9F726F899
:10C4200004900391514A524B09990E98F8F77AFFFC
:10C43000039B049AF9F7D0F91ED20220FEF72CFBD9
:10C44000FEF706FB49004908E20FD20711431BB073
:10C45000F0BD6A00474B52089A420DD3464AAA18CB
:10C46000024300D0CBE532463B46F8F7FFFF099B7D
:10C470000E9AF9F7B1F9F5D96800002340082C4964
:10C480000393020D3D4B5218984223DD0120000515
:10C49000521CD04042195000400D40183849794490
:10C4A000096813468C463749C1408B43120301216A
:10C4B000120B090551181422101AC1400391002DC6
:10C4C00001DA48420390624630463946F8F7CEFF1B
:10C4D00006460F4632463B4609990E98F8F722FF6A
:10C4E00000252A46284B28460591F8F7CDFF0791ED
:10C4F0000C90264A264B28460599F8F7C5FF00916F
:10C50000029032463B4628460599F8F7AFFF099B53
:10C510000E9AF8F7B1FF1F4A1F4BF8F7B5FF009BC3
:10C52000029AF8F7FFFE07460B460246099135E0EE
:10C5300001FCFFFF0000F03F8E9803007AB60B006D
:10C540006A070000AC070000D606000000000840A3
:10C5500009C7EE3FFD033ADCF5015B14E02F3EBE58
:10C56000AA0500007005000000009040FE822B65C7
:10C570004715973C00CC904000346F3F0000E03FEF
:10C58000C6040000FFFF0F00432EE63F396CA80CE5
:10C59000615C20BEEF39FAFE422EE63F07990C9807
:10C5A000F8F7C0FE05460E46079B0C9AF8F75EFFAB
:10C5B0003A46099BF8F760FF09912A4633460E90E8
:10C5C00010461946F8F760FF074602462F480B460B
:10C5D000059105217844FEF7CFF93A46059BF8F717
:10C5E00053FF2A463346F8F747FF0746019128468E
:10C5F0003146099B0E9AF8F747FF099B0E9AF8F708
:10C6000091FE012304910C9000229B07384601996A
:10C61000F8F72CFF05910E903A4628463146019BCB
:10C62000F8F732FF059B0E9AF8F796FF049B0C9AD9
:10C63000F8F71CFF2A463346F8F718FF0022144B80
:10C64000F8F71AFF064603980D460005411909152B
:10C65000002912DC30462946039AF8F7F5FFFEF769
:10C6600045F9042801D1FEF7FDF930462946039A21
:10C67000F8F7EAFF064601E004E029180B463246C7
:10C6800021460898F8F700FF1BB0F0BD68030000D2
:10C690000000F03FF0B58C46002510260521090763
:10C6A0008E620E4C08E067467F5DE760A768FF0773
:10C6B000FCD0E7681F706D1C8542F4DB0020074644
:10C6C00006E0E760A568ED07FCD0E5681D54401C56
:10C6D0009042F6D38E610020F0BD00000030014092
:10C6E00070B572B60124074DA40221462846F9F719
:10C6F0006DFC002804D0224603492846F9F70AFDBC
:10C7000062B670BD00FC0008C00D0020F8B50646FA
:10C710000C46F9F76FF9051E0F4600D001200143C2
:10C7200049000B484908411AC90F0DD0002E01D00D
:10C73000012100E000210C4361004908401AC00FAC
:10C7400002D10120FEF7A8F928463946F8BD0000BD
:10C750000000F07FF8B515460E460746002407E0B6
:10C760003819C0B200F008F8641C2870E4B26D1CDF
:10C77000B442F5D33046F8BD10B50446FBF79CFF34
:10C78000EE20FBF76CFFFBF7D0FF2046FBF767FFBF
:10C79000FBF7CBFFFBF790FFEF20FBF760FFFBF70A
:10C7A000C4FF0020FBF72EFF0446FBF7A0FF204646
:10C7B00010BD704770B50D460446FBF77DFFEE20B7
:10C7C000FBF74DFFFBF7B1FF2046FBF748FFFBF7F8
:10C7D000ACFF2846FBF743FFFBF7A7FFFBF787FFFC
:10C7E0000A20FEF7A2FA70BDF0B500251026052735
:10C7F0009C463F070B46BE620C4C06E0595DE1606B
:10C80000A168C907FCD0E1686D1C8542F6DB0020F9
:10C8100007E06146095CE160A168C907FCD0E168F6
:10C82000401C9042F5D3BE610020F0BD00300140B5
:10C830000000010203040005405C0000A05C04004D
:10C84000C06C0800805C0400E03F1E00E07D1E001C
:10C8500007A9022570889B880A00160001000600BF
:10C860000100020087008D002D001A3152001A339A
:10C870009A001A351D011A376B003B31BE003B335D
:10C880005E013B3596023B37000099599959EB51AF
:10C890008F421E45142E0080EB51F5283333E13AC8
:10C8A000703DE13AC235852BC2353333C235C235CE
:10C8B000AE47E13A5138A330513800000000000083
:10C8C00000000102030406070809030406080C100F
:10C8D00018203000000000010203040000000000E6
:10C8E000000000000000F03F000000000000F83FE2
:10C8F00000000000000000000000004003B8E23F1C
:10C90000000000000000000006D0CF43EBFD4C3ECD
:10C91000033333333333E33FFFAB6FDBB66DDB3FC2
:10C920004D268F515555D53F01411DA96074D13F0A
:10C9300065DBC9934A86CD3FEF4E454A287ECA3F04
:10C940003E5555555555C53F93BDBE166CC166BF86
:10C950002CDE25AF6A56113FF16BD2C541BDBBBE7F
:10C96000D0A4BE726937663E0000000000000000DF
:10C9700090C900080000002068010000BC5A0008AF
:10C98000D4C9000868010020001B000088AA000824
:10C990000124130704380D091E0805400826091054
:10C9A0004008560A131D043B08BE0516D8BC4010AB
:10C9B000085201033AC842077052030CE5800C1478
:10C9C0000202141509090102628149C8013A29408D
:04C9D000920492201B
:04000005080050C1DE
:00000001FF
